:020000040800F2
:10000000B1AA010000000000000000000000000094
:1000100000000000000000000000000000000000E0
:1000200000000000000000000000000000000000D0
:1000300000000000000000000000000000000000C0
:1000400000000000000000000000000000000000B0
:1000500000000000000000000000000000000000A0
:10006000000000008A4800080000000000000000B6
:100070000000000000000000000000000000000080
:100080000000000000000000000000000000000070
:100090000000000000000000000000000000000060
:1000A0000000000000000000000000000000000050
:1000B0000000000000000000000000000000000040
:1000C000D24800080000000000000000000000000E
:1000D0000000000000000000000000000000000020
:1000E0000000000000000000000000000000000010
:1000F000000000008C480008000000000000000024
:1001000000000000000000000000000000000000EF
:1001100000000000000000000000000000000000DF
:1001200000000000000000000000000000000000CF
:1001300000000000000000000000000000000000BF
:1001400000000000000000000000000000000000AF
:1001500000000000000000007448000873700430C4
:10016000170500001305C5FF8545F605637BB5003F
:1001700089816378B500170500001305C5002E9529
:1001800002859302002073A0027D970200009382F3
:1001900062E773907230979200009382A2E67390A8
:1001A000C27E73E0C07E979200009382A2DD7390BE
:1001B000523097110018938161CB178100181301F9
:1001C00061E417B50000130525AC97050018938569
:1001D00065E3170600181306664B63FAC500832211
:1001E000050023A0550011059105E3EAC5FE17059A
:1001F00000181305A549971500189385A550637736
:10020000B500232005001105E36DB5FE73F0023241
:10021000EF20E01601458145EF80504501A073E0D5
:0C0220000232828073F002328280000003
:100240000000000000000000010203040607080986
:100250000000000001000000020000000300000098
:10026000743D000828420008263D00089641000819
:10027000263D00082C410008B23E0008CC3F000893
:10028000D03F000820400008C4400008F8400008A3
:10029000284100082A3D00083C3D0008603D000858
:1002A0001003520056002D004C0049004E004B0038
:1002B00000000000220347004400330032005600D3
:1002C000460031003000330043002D00530054003D
:1002D00041005200540000002E0347004400330048
:1002E00032005800580058002D0033002E00300016
:1002F0002E0030002D0037007A00380078003900D9
:100300007900650072000000120100020200004046
:10031000E9288A01000101020301000080AC000805
:10032000A0020008B4020008D80200084744333293
:100330005646313033432D5354415254000000008F
:100340003C3F786D6C2076657273696F6E3D22312B
:100350002E30223F3E3C21444F4354595045207497
:1003600061726765742053595354454D2022676468
:10037000622D7461726765742E647464223E3C74ED
:1003800061726765742076657273696F6E3D2231A4
:100390002E30223E3C66656174757265206E616D1B
:1003A000653D226F72672E676E752E6764622E72CE
:1003B000697363762E637075223E3C726567206EAA
:1003C000616D653D227A65726F222062697473697E
:1003D0007A653D22333222207265676E756D3D224B
:1003E000302220736176652D726573746F72653D7E
:1003F000227965732220747970653D22696E7422BA
:100400002067726F75703D2267656E6572616C2240
:100410002F3E3C726567206E616D653D22726122E0
:100420002062697473697A653D22333222207265D5
:10043000676E756D3D22312220736176652D726580
:1004400073746F72653D22796573222074797065CB
:100450003D22696E74222067726F75703D22676558
:100460006E6572616C222F3E3C726567206E616D15
:10047000653D227370222062697473697A653D223A
:10048000333222207265676E756D3D2232222073F1
:100490006176652D726573746F72653D227965733F
:1004A0002220747970653D22696E74222067726F14
:1004B00075703D2267656E6572616C222F3E3C72DD
:1004C0006567206E616D653D2267702220626974E8
:1004D00073697A653D22333222207265676E756DCD
:1004E0003D22332220736176652D726573746F72BD
:1004F000653D227965732220747970653D22696EAD
:1005000074222067726F75703D2267656E65726137
:100510006C222F3E3C726567206E616D653D2274D2
:1005200070222062697473697A653D223332222019
:100530007265676E756D3D22342220736176652D7C
:10054000726573746F72653D2279657322207479C8
:1005500070653D22696E74222067726F75703D224E
:1005600067656E6572616C222F3E3C726567206E16
:10057000616D653D227430222062697473697A6509
:100580003D22333222207265676E756D3D22352221
:1005900020736176652D726573746F72653D227983
:1005A00065732220747970653D22696E742220671C
:1005B000726F75703D2267656E6572616C222F3EA9
:1005C0003C726567206E616D653D22743122206248
:1005D000697473697A653D22333222207265676ED1
:1005E000756D3D22362220736176652D72657374B8
:1005F0006F72653D227965732220747970653D22A2
:10060000696E74222067726F75703D2267656E6532
:1006100072616C222F3E3C726567206E616D653D94
:10062000227432222062697473697A653D22333202
:1006300022207265676E756D3D22372220736176C8
:10064000652D726573746F72653D22796573222022
:10065000747970653D22696E74222067726F7570BF
:100660003D2267656E6572616C222F3E3C72656744
:10067000206E616D653D2266702220626974736927
:100680007A653D22333222207265676E756D3D2298
:10069000382220736176652D726573746F72653DC3
:1006A000227965732220747970653D22696E742207
:1006B0002067726F75703D2267656E6572616C228E
:1006C0002F3E3C726567206E616D653D227331225D
:1006D0002062697473697A653D2233322220726523
:1006E000676E756D3D22392220736176652D7265C6
:1006F00073746F72653D2279657322207479706519
:100700003D22696E74222067726F75703D226765A5
:100710006E6572616C222F3E3C726567206E616D62
:10072000653D226130222062697473697A653D22D9
:10073000333222207265676E756D3D223130222082
:10074000736176652D726573746F72653D2279658C
:10075000732220747970653D22696E74222067725D
:100760006F75703D2267656E6572616C222F3E3C2D
:10077000726567206E616D653D226131222062697C
:100780007473697A653D22333222207265676E7513
:100790006D3D2231312220736176652D726573744F
:1007A0006F72653D227965732220747970653D22F0
:1007B000696E74222067726F75703D2267656E6581
:1007C00072616C222F3E3C726567206E616D653DE3
:1007D000226132222062697473697A653D22333264
:1007E00022207265676E756D3D2231322220736161
:1007F00076652D726573746F72653D22796573221B
:1008000020747970653D22696E74222067726F755D
:10081000703D2267656E6572616C222F3E3C726589
:1008200067206E616D653D226133222062697473B9
:10083000697A653D22333222207265676E756D3D9F
:100840002231332220736176652D726573746F7265
:10085000653D227965732220747970653D22696E49
:1008600074222067726F75703D2267656E657261D4
:100870006C222F3E3C726567206E616D653D226182
:1008800034222062697473697A653D2233322220F2
:100890007265676E756D3D22313422207361766515
:1008A0002D726573746F72653D22796573222074B1
:1008B0007970653D22696E74222067726F75703D94
:1008C0002267656E6572616C222F3E3C72656720FF
:1008D0006E616D653D226135222062697473697AAB
:1008E000653D22333222207265676E756D3D22317F
:1008F000352220736176652D726573746F72653D64
:10090000227965732220747970653D22696E7422A4
:100910002067726F75703D2267656E6572616C222B
:100920002F3E3C726567206E616D653D2261362207
:100930002062697473697A653D22333222207265C0
:10094000676E756D3D2231362220736176652D729A
:100950006573746F72653D227965732220747970B6
:10096000653D22696E74222067726F75703D226743
:10097000656E6572616C222F3E3C726567206E6108
:100980006D653D226137222062697473697A653D25
:1009900022333222207265676E756D3D2231372217
:1009A00020736176652D726573746F72653D22796F
:1009B00065732220747970653D22696E7422206708
:1009C000726F75703D2267656E6572616C222F3E95
:1009D0003C726567206E616D653D22733222206234
:1009E000697473697A653D22333222207265676EBD
:1009F000756D3D2231382220736176652D726573E5
:100A0000746F72653D227965732220747970653D3B
:100A100022696E74222067726F75703D2267656E61
:100A20006572616C222F3E3C726567206E616D6558
:100A30003D227333222062697473697A653D2233E3
:100A40003222207265676E756D3D22313922207326
:100A50006176652D726573746F72653D2279657379
:100A60002220747970653D22696E74222067726F4E
:100A700075703D2267656E6572616C222F3E3C7217
:100A80006567206E616D653D227334222062697452
:100A900073697A653D22333222207265676E756D07
:100AA0003D2232302220736176652D726573746F3A
:100AB00072653D227965732220747970653D2269E3
:100AC0006E74222067726F75703D2267656E657265
:100AD000616C222F3E3C726567206E616D653D2220
:100AE0007335222062697473697A653D223332223C
:100AF000207265676E756D3D2232312220736176FA
:100B0000652D726573746F72653D2279657322205D
:100B1000747970653D22696E74222067726F7570FA
:100B20003D2267656E6572616C222F3E3C7265677F
:100B3000206E616D653D227336222062697473698F
:100B40007A653D22333222207265676E756D3D22D3
:100B500032322220736176652D726573746F72650F
:100B60003D227965732220747970653D22696E7427
:100B7000222067726F75703D2267656E6572616CC9
:100B8000222F3E3C726567206E616D653D22733792
:100B9000222062697473697A653D223332222072A1
:100BA00065676E756D3D2232332220736176652D47
:100BB000726573746F72653D227965732220747952
:100BC00070653D22696E74222067726F75703D22D8
:100BD00067656E6572616C222F3E3C726567206EA0
:100BE000616D653D227338222062697473697A658C
:100BF0003D22333222207265676E756D3D2232349C
:100C00002220736176652D726573746F72653D2263
:100C10007965732220747970653D22696E74222093
:100C200067726F75703D2267656E6572616C222F09
:100C30003E3C726567206E616D653D2273392220EE
:100C400062697473697A653D223332222072656766
:100C50006E756D3D2232352220736176652D726589
:100C600073746F72653D22796573222074797065A3
:100C70003D22696E74222067726F75703D22676530
:100C80006E6572616C222F3E3C726567206E616DED
:100C9000653D22733130222062697473697A653D43
:100CA00022333222207265676E756D3D2232362204
:100CB00020736176652D726573746F72653D22795C
:100CC00065732220747970653D22696E74222067F5
:100CD000726F75703D2267656E6572616C222F3E82
:100CE0003C726567206E616D653D22733131222053
:100CF00062697473697A653D2233322220726567B6
:100D00006E756D3D2232372220736176652D7265D6
:100D100073746F72653D22796573222074797065F2
:100D20003D22696E74222067726F75703D2267657F
:100D30006E6572616C222F3E3C726567206E616D3C
:100D4000653D227433222062697473697A653D229D
:100D5000333222207265676E756D3D223238222053
:100D6000736176652D726573746F72653D22796566
:100D7000732220747970653D22696E742220677237
:100D80006F75703D2267656E6572616C222F3E3C07
:100D9000726567206E616D653D2274342220626940
:100DA0007473697A653D22333222207265676E75ED
:100DB0006D3D2232392220736176652D7265737420
:100DC0006F72653D227965732220747970653D22CA
:100DD000696E74222067726F75703D2267656E655B
:100DE00072616C222F3E3C726567206E616D653DBD
:100DF000227435222062697473697A653D22333228
:100E000022207265676E756D3D223330222073613A
:100E100076652D726573746F72653D2279657322F4
:100E200020747970653D22696E74222067726F7537
:100E3000703D2267656E6572616C222F3E3C726563
:100E400067206E616D653D2274362220626974737D
:100E5000697A653D22333222207265676E756D3D79
:100E60002233312220736176652D726573746F723F
:100E7000653D227965732220747970653D22696E23
:100E800074222067726F75703D2267656E657261AE
:100E90006C222F3E3C726567206E616D653D22704D
:100EA00063222062697473697A653D22333222209D
:100EB0007265676E756D3D223332222073617665EF
:100EC0002D726573746F72653D227965732220748B
:100ED0007970653D22696E74222067726F75703D6E
:100EE0002267656E6572616C222F3E3C2F666561DC
:100EF000747572653E3C66656174757265206E61DD
:100F00006D653D226F72672E676E752E6764622E67
:100F100072697363762E637372223E3C726567203A
:100F20006E616D653D226D7374617475732220620C
:100F3000697473697A653D22333222207265676E67
:100F4000756D3D223833332220736176652D7265CD
:100F500073746F72653D226E6F2220747970653DE7
:100F600022696E74222067726F75703D22637372FE
:100F7000222F3E3C726567206E616D653D226D6972
:100F80007361222062697473697A653D223332226B
:100F9000207265676E756D3D22383334222073618F
:100FA00076652D726573746F72653D226E6F2220B7
:100FB000747970653D22696E74222067726F757056
:100FC0003D22637372222F3E3C726567206E616D15
:100FD000653D226D6965222062697473697A653D99
:100FE00022333222207265676E756D3D22383337A9
:100FF0002220736176652D726573746F72653D2270
:101000006E6F2220747970653D22696E74222067AC
:10101000726F75703D22637372222F3E3C7265675A
:10102000206E616D653D226D747665632220626974
:101030007473697A653D22333222207265676E755A
:101040006D3D223833382220736176652D726573C9
:10105000746F72653D226E6F2220747970653D2237
:10106000696E74222067726F75703D2263737222FD
:101070002F3E3C726567206E616D653D226D636F2A
:10108000756E746572656E222062697473697A6523
:101090003D22333222207265676E756D3D223833F2
:1010A000392220736176652D726573746F72653DA8
:1010B000226E6F2220747970653D22696E74222041
:1010C00067726F75703D22637372222F3E3C7265AA
:1010D00067206E616D653D226D7363726174636834
:1010E000222062697473697A653D2233322220724C
:1010F00065676E756D3D22383937222073617665DC
:101100002D726573746F72653D226E6F2220747943
:1011100070653D22696E74222067726F75703D2282
:10112000637372222F3E3C726567206E616D653D70
:10113000226D657063222062697473697A653D224D
:10114000333222207265676E756D3D223839382240
:1011500020736176652D726573746F72653D226EC2
:101160006F2220747970653D22696E742220677247
:101170006F75703D22637372222F3E3C726567204B
:101180006E616D653D226D636175736522206269D4
:101190007473697A653D22333222207265676E75F9
:1011A0006D3D223839392220736176652D72657361
:1011B000746F72653D226E6F2220747970653D22D6
:1011C000696E74222067726F75703D22637372229C
:1011D0002F3E3C726567206E616D653D226D7476B1
:1011E000616C222062697473697A653D2233322210
:1011F000207265676E756D3D223930302220736133
:1012000076652D726573746F72653D226E6F222054
:10121000747970653D22696E74222067726F7570F3
:101220003D22637372222F3E3C726567206E616DB2
:10123000653D226D6970222062697473697A653D2B
:1012400022333222207265676E756D3D223930314E
:101250002220736176652D726573746F72653D220D
:101260006E6F2220747970653D22696E742220674A
:10127000726F75703D22637372222F3E3C726567F8
:10128000206E616D653D227473656C656374222008
:1012900062697473697A653D223332222072656710
:1012A0006E756D3D22323031372220736176652DA7
:1012B000726573746F72653D226E6F22207479704F
:1012C000653D22696E74222067726F75703D2263DE
:1012D0007372222F3E3C726567206E616D653D2200
:1012E000746461746131222062697473697A653D46
:1012F00022333222207265676E756D3D22323031A5
:10130000382220736176652D726573746F72653D46
:10131000226E6F2220747970653D22696E742220DE
:1013200067726F75703D22637372222F3E3C726547
:1013300067206E616D653D227464617461322220A4
:1013400062697473697A653D22333222207265675F
:101350006E756D3D22323031392220736176652DF4
:10136000726573746F72653D226E6F22207479709E
:10137000653D22696E74222067726F75703D22632D
:101380007372222F3E3C726567206E616D653D224F
:10139000746461746133222062697473697A653D93
:1013A00022333222207265676E756D3D22323032F3
:1013B000302220736176652D726573746F72653D9E
:1013C000226E6F2220747970653D22696E7422202E
:1013D00067726F75703D22637372222F3E3C726597
:1013E00067206E616D653D226463737222206269BD
:1013F0007473697A653D22333222207265676E7597
:101400006D3D22323033332220736176652D726553
:1014100073746F72653D226E6F2220747970653D22
:1014200022696E74222067726F75703D2263737239
:10143000222F3E3C726567206E616D653D226470AF
:1014400063222062697473697A653D2233322220F7
:101450007265676E756D3D223230333422207361C0
:1014600076652D726573746F72653D226E6F2220F2
:10147000747970653D22696E74222067726F757091
:101480003D22637372222F3E3C726567206E616D50
:10149000653D2264736372617463682220626974BB
:1014A00073697A653D22333222207265676E756DED
:1014B0003D22323033352220736176652D7265739B
:1014C000746F72653D226E6F2220747970653D22C3
:1014D000696E74222067726F75703D226373722289
:1014E0002F3E3C726567206E616D653D226D6379AC
:1014F000636C65222062697473697A653D223332B8
:1015000022207265676E756D3D2232383831222097
:10151000736176652D726573746F72653D226E6FAF
:101520002220747970653D22696E74222067726F83
:1015300075703D22637372222F3E3C726567206E88
:10154000616D653D226D696E7374726574222062EF
:10155000697473697A653D22333222207265676E41
:10156000756D3D22323838332220736176652D72D5
:101570006573746F72653D226E6F22207479706599
:101580003D22696E74222067726F75703D2263730D
:1015900072222F3E3C726567206E616D653D226D43
:1015A0006379636C6568222062697473697A653D4A
:1015B00022333222207265676E756D3D22333030E2
:1015C000392220736176652D726573746F72653D83
:1015D000226E6F2220747970653D22696E7422201C
:1015E00067726F75703D22637372222F3E3C726585
:1015F00067206E616D653D226D696E7374726574EE
:1016000068222062697473697A653D223332222030
:101610007265676E756D3D22333031312220736102
:1016200076652D726573746F72653D226E6F222030
:10163000747970653D22696E74222067726F7570CF
:101640003D22637372222F3E3C726567206E616D8E
:10165000653D226379636C65222062697473697ADF
:10166000653D22333222207265676E756D3D2233EF
:101670003133372220736176652D726573746F7212
:10168000653D226E6F2220747970653D22696E740B
:10169000222067726F75703D22637372222F3E3C69
:1016A000726567206E616D653D2274696D652220EB
:1016B00062697473697A653D2233322220726567EC
:1016C0006E756D3D22333133382220736176652D7E
:1016D000726573746F72653D226E6F22207479702B
:1016E000653D22696E74222067726F75703D2263BA
:1016F0007372222F3E3C726567206E616D653D22DC
:10170000696E7374726574222062697473697A6594
:101710003D22333222207265676E756D3D22333172
:1017200033392220736176652D726573746F72652B
:101730003D226E6F2220747970653D22696E74229D
:101740002067726F75703D22637372222F3E3C7268
:101750006567206E616D653D226379636C65682203
:101760002062697473697A653D2233322220726582
:10177000676E756D3D223332363522207361766592
:101780002D726573746F72653D226E6F22207479BD
:1017900070653D22696E74222067726F75703D22FC
:1017A000637372222F3E3C726567206E616D653DEA
:1017B0002274696D6568222062697473697A653D77
:1017C00022333222207265676E756D3D22333236C8
:1017D000362220736176652D726573746F72653D74
:1017E000226E6F2220747970653D22696E7422200A
:1017F00067726F75703D22637372222F3E3C726573
:1018000067206E616D653D22696E737472657468E0
:10181000222062697473697A653D22333222207214
:1018200065676E756D3D22333236372220736176DF
:10183000652D726573746F72653D226E6F22207420
:101840007970653D22696E74222067726F75703DF4
:1018500022637372222F3E3C726567206E616D6554
:101860003D226D76656E646F7269642220626974D0
:1018700073697A653D22333222207265676E756D19
:101880003D22333932322220736176652D726573C1
:10189000746F72653D226E6F2220747970653D22EF
:1018A000696E74222067726F75703D2263737222B5
:1018B0002F3E3C726567206E616D653D226D6172E1
:1018C00063686964222062697473697A653D2233B2
:1018D0003222207265676E756D3D223339323322B4
:1018E00020736176652D726573746F72653D226E2B
:1018F0006F2220747970653D22696E7422206772B0
:101900006F75703D22637372222F3E3C72656720B3
:101910006E616D653D226D696D706964222062693A
:101920007473697A653D22333222207265676E7561
:101930006D3D22333932342220736176652D726514
:1019400073746F72653D226E6F2220747970653DED
:1019500022696E74222067726F75703D2263737204
:10196000222F3E3C726567206E616D653D226D6879
:101970006172746964222062697473697A653D22B8
:10198000333222207265676E756D3D2233393235F0
:101990002220736176652D726573746F72653D22C6
:1019A0006E6F2220747970653D22696E7422206703
:1019B000726F75703D22637372222F3E3C2F6665F5
:1019C00061747572653E3C66656174757265206E02
:1019D000616D653D226F72672E676E752E6764625A
:1019E0002E72697363762E7669727475616C223E0D
:1019F0003C726567206E616D653D2270726976226A
:101A00002062697473697A653D22382220726567A5
:101A10006E756D3D22343136312220736176652D2D
:101A2000726573746F72653D226E6F2220747970D7
:101A3000653D22696E74222067726F75703D226762
:101A4000656E6572616C222F3E3C2F666561747510
:101A500072653E3C2F7461726765743E0000000041
:101A60004744333256463130330000003C6D656DDB
:101A70006F72792D6D61703E3C6D656D6F7279206E
:101A8000747970653D2272616D2220737461727485
:101A90003D223078303030303030303022206C65AC
:101AA0006E6774683D223078383030303030302204
:101AB0002F3E3C6D656D6F727920747970653D22A3
:101AC000666C617368222073746172743D22307891
:101AD000303830303030303022206C656E677468BA
:101AE0003D2230783230303030223E3C70726F70A0
:101AF00065727479206E616D653D22626C6F636BF7
:101B000073697A65223E30783430303C2F70726FC2
:101B100070657274793E3C2F6D656D6F72793E3CD5
:101B20006D656D6F727920747970653D2272616D9B
:101B3000222073746172743D223078303830323034
:101B400030303022206C656E6774683D22307866D4
:101B500037666530303030222F3E3C2F6D656D6F1B
:101B600072792D6D61703E002530327800000000E2
:101B7000F88C0008448E0008448E0008448E00084B
:101B8000448E0008448E0008448E0008448E0008ED
:101B9000448E0008448E0008448E0008448E0008DD
:101BA000448E0008448E0008448E0008448E0008CD
:101BB000448E0008448E0008448E0008448E0008BD
:101BC000448E0008448E0008448E0008448E0008AD
:101BD000448E0008448E0008448E0008448E00089D
:101BE000448E0008448E0008448E0008448E00088D
:101BF000448E0008448E0008448E0008448E00087D
:101C0000448E0008448E0008448E0008448E00086C
:101C1000448E0008448E0008448E0008448E00085C
:101C2000448E0008448E0008448E0008448E00084C
:101C3000448E0008448E0008448E0008448E00083C
:101C4000448E0008448E0008448E0008448E00082C
:101C5000448E0008448E0008448E0008448E00081C
:101C6000448E0008448E0008448E0008448E00080C
:101C7000448E0008448E0008448E0008448E0008FC
:101C8000448E0008448E0008448E0008448E0008EC
:101C9000448E0008448E0008448E0008448E0008DC
:101CA000448E0008448E0008448E0008448E0008CC
:101CB000448E0008448E0008448E0008448E0008BC
:101CC000448E0008448E0008448E0008448E0008AC
:101CD000448E0008448E0008448E0008448E00089C
:101CE000448E0008448E0008448E0008448E00088C
:101CF000448E0008448E0008448E0008448E00087C
:101D0000448E0008448E0008448E0008448E00086B
:101D1000448E0008448E0008448E0008448E00085B
:101D2000448E0008448E0008448E0008448E00084B
:101D3000448E0008448E0008E28A0008448E0008A1
:101D4000448E0008448E0008448E0008448E00082B
:101D5000448E0008448E0008448E0008448E00081B
:101D6000448E0008448E0008448E0008448E00080B
:101D7000448E0008228C0008448E0008448E00081F
:101D8000448E0008448E0008448E0008448E0008EB
:101D9000608C0008448E0008448E0008448E0008C1
:101DA000448E0008448E0008448E0008448E0008CB
:101DB000448E0008A48C0008448E0008448E00085D
:101DC000448E0008448E0008448E0008448E0008AB
:101DD000448E0008F68A0008448E0008448E0008ED
:101DE000168B0008448E0008448E0008448E0008BC
:101DF000EA8C0008448E0008128D0008448E00080A
:101E0000288D0008448E00083E8D0008448E00088E
:101E1000548D0008448E00086A8D0008448E000826
:101E2000808D0008448E0008968D0008448E0008BE
:101E3000AC8D0008448E0008C28D0008448E000856
:101E4000D88D0008448E0008EE8D0008448E0008EE
:101E5000048E0008448E00081A8E0008448E000884
:101E6000308E0008448E0008BA8B000825780000E8
:101E70005153746172744E6F41636B4D6F646500B2
:101E80005A25782C25782C25780000007153757020
:101E9000706F727465643A0071586665723A66656F
:101EA0006174757265733A726561643A74617267E0
:101EB00065742E786D6C3A0071586665723A6D657E
:101EC0006D6F72792D6D61703A726561643A3A0096
:101ED0007152636D642C00007265736574000000BC
:101EE00068616C74000000003A2820756E7375708C
:101EF000706F72746564206D6F6E69746F722063A9
:101F00006F6D6D616E64210A000000005330320075
:101F100076466C61736845726173653A0000000033
:101F200076466C61736857726974653A0000000008
:101F300076466C617368446F6E650000764D75730C
:101F4000745265706C79456D707479007A25782CBF
:101F500025782C25780000000A52562D4C494E4B0E
:101F6000204552524F523A2074686520746172675E
:101F70006574206973206E6F7420636F6E6E656385
:101F8000746564210A0000000A52562D4C494E4BDC
:101F9000204552524F523A2074686520746172672E
:101FA0006574206973206E6F7420737570706F7222
:101FB0007465642C20757067726164652052562DBB
:101FC0004C494E4B206669726D77617265210A003B
:101FD0000A52562D4C494E4B204552524F523A20F0
:101FE000736F6D657468696E672077726F6E6720B6
:101FF00077697468206465627567206D6F64756CBD
:1020000065210A000A52562D4C494E4B204552522A
:102010004F523A20756E6B6E6F776E206572726FDD
:1020200072210A0052562D4C494E4B2076302E31EB
:102030003A2000002C20636F6E6669676564206635
:102040006F7220002066616D696C792E0A000000B5
:1020500054303200543035004525303278000000CD
:102060004F4B00005061636B657453697A653D3472
:1020700030353B5153746172744E6F41636B4D6FD9
:1020800064652B3B71586665723A6665617475725A
:1020900065733A726561642B3B71586665723A6D7F
:1020A000656D6F72792D6D61703A726561642B0098
:1020B00000010202030303030404040404040404EF
:1020C00005050505050505050505050505050505C0
:1020D00006060606060606060606060606060606A0
:1020E0000606060606060606060606060606060690
:1020F0000707070707070707070707070707070770
:10210000070707070707070707070707070707075F
:10211000070707070707070707070707070707074F
:10212000070707070707070707070707070707073F
:10213000080808080808080808080808080808081F
:10214000080808080808080808080808080808080F
:1021500008080808080808080808080808080808FF
:1021600008080808080808080808080808080808EF
:1021700008080808080808080808080808080808DF
:1021800008080808080808080808080808080808CF
:1021900008080808080808080808080808080808BF
:1021A00008080808080808080808080808080808AF
:1021B000232D302B20000000686C4C0065666745BD
:1021C00046470000303132333435363738394142F2
:1021D0004344454600000000303132333435363751
:1021E000383961626364656600000000412D466114
:1021F0002D66383930313233343536375D000000E2
:102200002B2D000030300000785800000000000046
:1022100000000000000000000000000000000000BE
:1022200000000000000000000000000000000000AE
:10223000000000000000000000000000000000009E
:10224000000000000000000000000000000000008E
:10225000000000000000000000000000000000007E
:10226000000000000000000000000000430000002B
:10227000504F5349580000002E000000002020203D
:102280002020202020202828282828202020202026
:1022900020202020202020202020202020881010F6
:1022A0001010101010101010101010101004040452
:1022B0000404040404040410101010101010414110
:1022C00041414141010101010101010101010101FE
:1022D0000101010101010101101010101010424212
:1022E00042424242020202020202020202020202CE
:1022F000020202020202020210101010200000006E
:1023000000000000000000000000000000000000CD
:1023100000000000000000000000000000000000BD
:1023200000000000000000000000000000000000AD
:10233000000000000000000000000000000000009D
:10234000000000000000000000000000000000008D
:10235000000000000000000000000000000000007D
:10236000000000000000000000000000000000006D
:10237000000000000000000000000000000041110B
:1023800006C6912C1305700599286122B2404101BF
:102390008280828001A08567FD176303F50001A09C
:1023A000411106C6C53F01A0B707002003A78766F5
:1023B0003A95B717002093870770636EF500B787CB
:1023C00000209387078063EAA700B707002023A4B3
:1023D000A7663A8582807D57EDBF7D57DDBFB70781
:1023E00000D223800700A38507001205B71700D28B
:1023F0003E9563F6A70023A00700C107DDBF8280DA
:102400000A05B71700D285073E9585472300F500DA
:1024100082800A05B71700D28D073E952300B500CC
:1024200082800A05B71700D28D073E950345050047
:102430008280B70700D22380A7008280B70700D22E
:1024400003C507008280411106C622C40605137425
:10245000F50FED371375150E7988418DD93FB240D0
:10246000224441018280411106C6C93F05813D8950
:10247000B24041018280411106C622C426C24AC030
:102480002A892E84CD37AA84914763F3A70091440B
:10249000A147858F3314F4001374F40F4A85513724
:1024A000B315950093F5F50FB3D5954093F5F50F5A
:1024B000C18D4A85B93FB24022449244024941014C
:1024C0008280411106C622C426C24AC02A892E84AF
:1024D000593F8D4763FAA70001442285B240224448
:1024E0009244024941018280AA8412041374F40FB9
:1024F0004A85053FA145B3849540B355954093F572
:10250000F50FB395950093F5F50FC18D4A851137F9
:10251000E9B7F327503093F707FC93E73700739040
:1025200057308280371702401C43C166D58F1CC3C9
:10253000814785073717024018439316E70063C6A3
:10254000060041677D17E396E7FEB71702409C43FC
:102550001397E7006343070001A0B7170240D84371
:10256000D8C3D843D8C3D84313670740D8C3D84388
:10257000B706C4DFFD16758FD8C3D843B7061D2034
:10258000558FD8C3D857BD76758FD8D7D85713670E
:102590001700D8D79843B7060001558F98C3B717CF
:1025A00002409C4313976700E35B07FEB7170240A6
:1025B000D843719BD8C3D84313672700D8C3B71734
:1025C0000240DC43A18BE5DF8280411106C6993FC2
:1025D000B24041018280411106C6B71702409843BC
:1025E0001367170098C3D843B706FFE0B106758F8D
:1025F000D8C39843B706F7FEFD16758F98C3984366
:10260000B706FCFFFD16758F98C3D843B70601DFE8
:10261000FD16758FD8C323A607029843B706F7EABD
:10262000FD16758F98C33707FF0098C7793FB240F2
:102630004101828093F8F50093F7050199C3B3E84F
:10264000C800814731A058C910C18507C207C1839E
:102650001D476360F70405473317F700758F75D77B
:1026600003230500139827003D4633160601134641
:10267000F6FF33766600339808013366C800130806
:102680008002E38205FD13088004E39F05FB18C95F
:1026900065BFA14731A050C958C18507C207C18392
:1026A0003D476363F70405463316F600758E75D60D
:1026B000032345003707004061173E970A073D484E
:1026C0003318E8001348F8FF337868003397E800C0
:1026D0003367070113088002E38F05FB13088004AA
:1026E000E39C05FB10C94DBF82800CC982804CC998
:1026F00082809357650037170240BA979843854602
:10270000B396A600558F98C38280935765003717FC
:102710000240BA9798438546B396A600558F98C352
:10272000828013576500B71702403E9714438547D0
:10273000B397A70093C7F7FFF58F1CC38280B71626
:102740000240DC42370740FF7D17F98F5D8DC8C21C
:1027500082800111B7070008938707249043D44370
:102760009847DC4732C836CA3ACC3ECE03A78181AF
:102770003AC493878181DC433EC63AC03EC2B71754
:102780000240DC4389838D8B09476381E706B716D6
:102790007A0093860620371602405C429183BD8BF7
:1027A0001810BA9703C707FF33D7E6005C42A1832E
:1027B0009D8B0C10AE9783C787FEB355F7005C4224
:1027C000AD839D8B1010B29783C707FEB357F700F8
:1027D00005466305C50C69C509476305E50C0D474A
:1027E0006303E50081473E8505618280B71702409B
:1027F000DC431397F700635C0708B7170240DC5708
:102800001397F70063500708B7160240D856118394
:102810003D8B93071700D456A18213F7F600930659
:1028200027004547638EE60437177A001307072011
:102830003357F7023307D702B7170240D457BD8A80
:1028400085063357D702B7160240DC42C983BD8BD9
:10285000D442139626006354060093E70701B94655
:1028600063ECF6028907B386E7023D46E395C7F2BB
:1028700093171700BA97939617000583BA9621BF4E
:10288000D1465DB737177A001307072075B737179A
:102890003D001307079045BF8507F1B7BA87A1B779
:1028A000B68791B7AE8781B7411106C6B71700400A
:1028B000938707C0630EF508B7170040938707C0DA
:1028C00063E5A702B7070040938707406304F50656
:1028D000B7170040938707806305F506B7070040E8
:1028E0006303F504B24041018280B717004093872B
:1028F00007406306F506B7370140938707C0630DAD
:10290000F500B7170040E31FF5FC13054040F53B09
:10291000130540403935F9B71305B030FD331305C1
:10292000B0300135C1B713050040C5331305004071
:10293000CD3B4DBF13051040C93B13051040D533A7
:1029400055B713052040D13313052040D93B59BF5B
:10295000130530405D3B13053040E13361B713058B
:1029600050406533130550406D3BADBF83D7050024
:102970001CD5B7370140938707C06300F504B7073C
:102980000040630CF502938707406308F502B71710
:102990000040938707806302F502B71700409387D2
:1029A00007C0630CF5001C41BD9B1CC11C4103D733
:1029B0004500418BD98F1CC115A01C4193F7F7F836
:1029C0001CC11C4103D7250013770706D98F1CC1F2
:1029D0001C4103D74500418BD98F1CC19C455CD558
:1029E000B71700406301F50293870740630DF500B8
:1029F0001C4193F7F7CF1CC11C4103D7C5001377C7
:102A00000730D98F1CC1B7370140938707C06307D0
:102A1000F5005C4993E717005CC9828083C7E50035
:102A20001CD9C5BF1C4193E717001CC182801C4103
:102A3000F99B1CC182801C41F59B1CC1828091477F
:102A40006387F50081E51C41ED9B1CC182801C4120
:102A500093E747001CC182805C45DD8D4CC58280B8
:102A60001C49FD8D99C1054582800145828093C531
:102A7000F5FF0CC98280F36704308280411106C6DD
:102A80001375F50FC932B24041018280411106C66B
:102A900022C426C24AC02A842E89B2849532CA85AD
:102AA0002285D13AA6852285293CB240224492440F
:102AB000024941018280B707014083A607401347BE
:102AC000F5FFF98E23A0D74083A64740F98E23A2B5
:102AD000D74083A68740F98E23A4D74083A6C7405A
:102AE000F98E23A6D74081CD85476382F5028547BD
:102AF0006304F6040DC68947630DF6048280B706A9
:102B0000014083A70640C98F23A0F640CDB7B70682
:102B1000014083A74640C98F23A2F640C9BFB7072B
:102B2000014083A68740558D23A4A74083A6C740B4
:102B3000758F23A6E7408280B707014083A68740B0
:102B4000758F23A4E74003A7C740598D23A6A7404C
:102B50008280B707014003A78740498F23A4E7403D
:102B600003A7C740598D23A6A7408280370701409D
:102B7000832707405D8D2320A7408280B70701404F
:102B800023AAA7408280B77700409843719B98C3DF
:102B90009843598D88C3F3E7108191E57300501075
:102BA000F3F710818280F3770430F3E7008173003C
:102BB0005010F3F70081F3670430DDB7411106C60A
:102BC00018411C4B93E717001CCB1C419C4B858B79
:102BD000EDFF0D45EF105043B240410182800111DD
:102BE00006CE22CC26CA4AC84EC652C456C25AC0C5
:102BF000230205008947A300F5002300C50011C684
:102C00008547630CF6080545CDA0B1472301F500C3
:102C10009947A301F5008947A302F500370904404D
:102C20002E84AA8485472303F500A303F500856756
:102C3000138B07804A9B930A0940130A0944938720
:102C400007E0B309F9001306C00B81452285EF6048
:102C50003007232024012322640123245401232C40
:102C60004407232C340B014783C734006373F704F4
:102C700093175700CA97856693850690BE951316DD
:102C8000270022964CC6938606B0B6979306870017
:102C90008A06A296DCC20507C1BFA1472301F50041
:102CA0009147A301F5008947A302F50037090050B9
:102CB00085BF814703C7240063F8E7029396570056
:102CC000CA96938606501387C7000A07229754C7EF
:102CD0009396C700CA960567BA961387C7010A0775
:102CE000229754C78507F9B70145F2406244D244A0
:102CF0004249B249224A924A024B0561828001113F
:102D000006CE22CC2AC42EC632841C42985F984735
:102D1000799B98C70347D1008547630DF702184296
:102D20005C4793E707045CC73285493D8347E10070
:102D3000A1EB37072D001C4098DF5145EF10B02D57
:102D40000347C10085476300F7040145F240624430
:102D5000056182801C423707100098DF1442DC4670
:102D60003707E0FF1307F7FBF98FDCC61442DC4698
:102D70003707F0FF7D17F98FDCC632858135C9B77B
:102D800037073D004DBF18401C4793E707021CC79B
:102D900018401C47859B1CC718401C4793E7A70099
:102DA0001CC765B78D06898271060A062A964846B1
:102DB0001386F6FF9DC283C7050003C715002207CF
:102DC000D98F03C725004207D98F03C73500620793
:102DD000D98F1CC19105B286E1BF014582800D06E5
:102DE0000982685D1307F6FF15C21C412380F500B8
:102DF00093D68700A380D50093D607012381D50001
:102E0000E183A381F50091053A86E9BF2E85828092
:102E1000411106C69A051C4193E505028CCB1C4165
:102E20009C4B93F70702E5FF0D45EF10F01D0145A0
:102E3000B24041018280411106C61C41414798CBF6
:102E40001C419C4BC18BEDFF0D45EF10F01B014564
:102E5000B240410182801C457D57D8C31845B70751
:102E600000C0FD175CCB1845B7170080938707801B
:102E70001CCF8347450091E718451C4F93E7070196
:102E80001CCF14459C4E37370C002907D98F9CCE98
:102E900018451C4793E717001CC701458280411164
:102EA00006C622C426C22A841445DC46370700A081
:102EB0007D17F98FDCC618455C47B7060040D58FF3
:102EC0005CC78327050C23A0070054459C427977F3
:102ED0001307F77FF98F9CC25C45984398C3584508
:102EE0001C43F19B1CC30347050085476307F7029A
:102EF00093048400C1452685213F26852D3F5C44EF
:102F000023A807005C4423AA07005C447D5798CFA0
:102F10005C4423AE0700814779A058451C4393E7E2
:102F200037001CC31C4513070008D8D31845B70742
:102F30004000938707081CD79305000805478D4775
:102F4000E3E8E7FA9306F7FFB7B70008938747C7A8
:102F50008606BE9683D60600B69593161700B697DA
:102F600083D70700C2071444CD8F1306F7030A0660
:102F7000B296DCC20507E1B7144337060048D18E8C
:102F800014C33DA8144337060048D18E14C31387D9
:102F900087000A072297544723A80600584793063C
:102FA000F00F14C785070347340063F0E704139755
:102FB00027002297584B1443E3C006FC2320070048
:102FC000139727002297544B23A80600584B9306CB
:102FD000F00F14C7138787000A0722975847144336
:102FE000E3C206FA232007005DB72285AD3501450F
:102FF000B240224492444101828058455C4393E7A9
:1030000027005CC3828058455C43F59B5CC382808B
:1030100058451C4393F7F7801CC358451C43920541
:10302000CD8F1CC38280411102C69C41BD8B3E885E
:1030300003870500634C0706138787000A072A9752
:103040005847138607018546B396C60036C6144313
:1030500013960601634406041443370634FC130632
:103060000680F18E14C3631C08045445944613F87B
:1030700066001043B7B60008938606C7C29683C69B
:103080000600D18E14C3144303C615004A06DA079E
:10309000D18FDD8EB7870010DD8E14C3B246584540
:1030A0005C4FD58F5CCF014541018280139727008B
:1030B0002A97584B8546B396F60036C649BF144347
:1030C00003D64500D18E14C37DBF9C41BD8B0387C1
:1030D0000500634807029386070105473317D700A9
:1030E000A1078A07AA97D0471C42E176FD16F58F03
:1030F0001CC25445DC4E1347F7FF7D8FD8CE0145E7
:10310000828005473317F7008A07AA97D04B1C42E5
:10311000E176FD16F58F1CC2E9BF011106CE904184
:103120003D8A93172600AA97DC4B98433AC69C4BDE
:103130003EC4A247370700E0F98F3EC4DC45BDE33B
:10314000A24737070800D98F3EC493172600AA97D5
:10315000DC4B224798CB034745008547630AF708B5
:1031600003C715008547630CF708B247370700848B
:10317000D98F3EC693172600AA97DC4B324798C3D7
:1031800003C715008547630DF708DC4581CB54451F
:10319000DC5A05473316C700D18FDCDA0145F2400F
:1031A000056182801DEA03D745006373F700BA8783
:1031B000DCC5A24737070800D98F3EC4DC4522474B
:1031C000D98F3EC403C715008547E310F7F8A2471F
:1031D00037070060D98F3EC48DBF03D74500BA972B
:1031E000FD17B3D7E702CE072247D98F3EC4F9B700
:1031F00093172600AA97DC4B984DD8CB95B75C4522
:103200009C4793F7071099C7B24737070020D98F1B
:103210003EC6A1BFB24737070010D98F3EC6B1B72F
:1032200083D6C5008C452105B53E8DBF9C41BD8B25
:10323000138787000A072A970328C7000326080078
:1032400003270801370300E03373670083A8C50034
:103250006383080095EF03D7450033676700B7061F
:103260000800558F2328E800834645000547638FF3
:10327000E60283C6150005476382E604370700842B
:10328000598EA1078A07AA97DC4790C3014582801F
:1032900083D64500B698FD18B3D8D80213973801E5
:1032A00033676700B3861603558F6DBF138787009A
:1032B0000A072A975847944D54CB65BF03C735007A
:1032C00009C737070020598E55BF37070010598EA0
:1032D00075B79C41BD8B03870500634D0700A107AF
:1032E0008A07AA97D8471C43B7062000D58F1CC36E
:1032F000014582808A07AA97DC4B3E879443E3D43A
:1033000006FE944337060040D18E94C3E9BF9C412A
:10331000BD8B0387050063460702A1078A07AA97AA
:10332000D4479C423707E0FF7D17F98F9CC283C7C3
:103330001500F91793F7F70F05476378F700014574
:1033400082808A07AA97D44BE9BF9C4237070010B6
:10335000D98F9CC2EDB75C45884FDC4F7D8D418194
:103360001375F5038280A1058A05AA95DC45984767
:103370005C45C84B798D82805C45884FDC4F7D8DE4
:103380001375F50382805845144B5C5BB3D7B700C7
:103390009E0793F7F70FD58F8A052E955849084752
:1033A0007D8D82805855B7070860E1071CCB034725
:1033B000450085476303F7008280130745425C554B
:1033C000D8CB58551C43B7860080D58F1CC3EDB7AA
:1033D0008347750091CB5C459C47858B91C703273C
:1033E000050C1C43F19B1CC3828018455C4B858BEC
:1033F00063950712411106C622C426C2404B1C4FDA
:103400007D8C79C0AA849317C40063C4070C9317FA
:10341000D40063C2070C856793870780E18FDDEFD7
:103420006341040C9377240081C79C440947D8CB9F
:1034300093778400B9C383A704439C4F99C326851F
:103440008297B707002083C7876893F7F70F9DC35C
:10345000B70700209387876803C70700050713771E
:10346000F70F2380E70083C7070093F7F70F09479B
:103470006364F7089C442147D8CB93770401C9E7DC
:103480009317340163C507089317240163C4070821
:103490009317B40063DC070083A70443DC4F99C390
:1034A000268582979C4437071000D8CB9317A40039
:1034B00063DC070083A704439C5399C32685829746
:1034C0009C4437072000D8CBB240224492444101AB
:1034D0008280A9202DBF26851D2235BF2685CD2EB1
:1034E00081B783C7740C93F7F70F2383F40C9C44C4
:1034F00037070080D8CB3DB72685EF00B071B707FE
:10350000002023840768BDB72685692295BF2685DC
:10351000A5249DBF2685A926A5BF8280797106D6E0
:1035200022D426D24AD04ECE2A8935352A848144E7
:10353000A1A0938784008A07CA97DC479C4B3EC6AC
:1035400013973400058F93172700CA9703D70727CF
:10355000B246370608007D16F18E158F23AEE7269A
:10356000A1A0A1EC0347C94299476318F7044A8513
:10357000153DA1A0058085043DC893771400FDDBAF
:1035800093F9F40FCE854A85F93B2AC4A247858B6F
:103590008DC7938784008A07CA97D84785471CC779
:1035A00003474900E307F7F8CE854A85EF00506DE1
:1035B000034749008547E306F7FAA247A18BDDDB05
:1035C000D5F8B707002083C7876893F7F70FDDD3D7
:1035D0004A85EF003064B70700202384076893878B
:1035E00084008A07CA97DC47214798C761B7054519
:1035F000B250225492540259F24945618280797145
:1036000006D622D426D24AD04ECE52CC2A89AD3309
:103610002A8481441DA893972400CA97DC4B054A4D
:1036200023A44701CE854A85EF00307383474900C4
:10363000639A470385E80347C94295476314F70235
:103640004A858D3305A00580850405CC9377140049
:10365000FDDB93F9F40FCE854A8535332AC6B24790
:10366000858BD5FBB24793F70708F1DFA6854A851E
:10367000F52493972400CA97DC4B1307000898C7DA
:10368000D9B70545B250225492540259F249624AC0
:1036900045618280797106D622D426D24AD04ECE98
:1036A00052CCAA8402C618451C4FBD9B1CCF1C459A
:1036B0009C533EC632491379F90032461182137485
:1036C000F67FB247BD8313F73700B247C583BD8B82
:1036D00089466383D70299466389D70498441C4F6F
:1036E00093E707011CCF0545B2502254925402596A
:1036F000F249624A4561828075D0131A3900B307D6
:103700002A4193992700AA99228683A54927210552
:10371000EFF0EFEC83A74927A29723AAF92603A687
:10372000C927229623AEC92655BF93163900B38602
:10373000264193972600AA9783C7C726BD8BD9FF3A
:10374000A147E31DF4F859FB228693054542210564
:10375000EFF0EFE893173900B3862741139726005F
:1037600026970326C7272296232EC726B7070020B1
:1037700005472384E7689DB7411106C622C426C2C7
:103780004AC02A8458455C43F99B5CC381452105A6
:10379000EFF00FE80147834734006371F702931796
:1037A0002700A297DC4B9306F00F94C7930787007E
:1037B0008A07A297DC4794C70507F1BF5C447D5791
:1037C00098CF5844C16785075CCF5C442547D8CB68
:1037D0005C44854484CB58441C4393F7F7801CC356
:1037E000A302040C22857D3E1C440567D8CB23260A
:1037F000042623280426232A0426232C0426232EE9
:103800000426232004282322042813090004231853
:1038100024279305C4262285EFF0FF802324040C7F
:103820002326040C2328040C232A040C232C040C28
:10383000232E040C2320040E930700F82304F40C19
:103840002316240D9305840C2285EFF0CFFD23036E
:10385000940C0545B24022449244024941018280C1
:1038600054459C46858313F73700DC4293F7F7EF06
:10387000DCC25445DC4293E70710DCC210455C46CD
:10388000F1769386F63FF58F5CC6B7B7000893874D
:10389000C7C7BA9703C707008D476301F702894777
:1038A000A300F5001445DC46056713070740D98FD0
:1038B000DCC61C450967D8CB05458280A300F5000E
:1038C0001445DC46096713070740D98FDCC6D5B716
:1038D000011106CE22CC2A8483477500A307F1008C
:1038E0005C459C47858B2307F1008347650C93F764
:1038F000F70F0D476387E7048147A306F10083476D
:10390000640C93F7F70FA303F40C91472303F40C13
:103910008347F10093F7F70F99CB8347E10093F7C3
:10392000F70F91C78347D10093F7F70F89EF18443A
:103930008567938707805CCB0545F240624405614B
:10394000828085475DBF0327040C1C4393E7370043
:103950001CC381450545EFF00FA3D1BF011106CE71
:1039600022CC26CA4AC84EC652C4AA892E891397A9
:1039700035000D8F93172700AA9703A7470D83A63D
:10398000870D158F03DAC70C6363EA003A8A0D0AC4
:10399000135A2A00A9A0138A3400135A2A00931735
:1039A0003900B3872741139427004E94939604015E
:1039B000C1821376F90F8325040D13858900EFF07A
:1039C0006FBE8327040DA6972328F40C8327840D4C
:1039D000BE94232C940C8327440D6386F404931720
:1039E0002900CE97DC4B9C4FC207C1836378FA0451
:1039F000131739003307274193172700CE9703A7E2
:103A0000870D83A7470D637BF702998F93163900C3
:103A1000B3862641139726004E978354C70CE3ECD8
:103A2000F4F6BE848DBF83A6C900D85A8547B397E4
:103A3000270193C7F7FFF98FDCDA55B70545F24048
:103A40006244D2444249B249224A0561828041110E
:103A500006C603C7250003C8450083C75500A20753
:103A600033E8070193178701E18763C3070613163D
:103A70003700B306E64093972600BE869387072655
:103A8000AA97B107AA9603C6C6261376F607238619
:103A9000C6263D8B83C60700C19A558F2380E70059
:103AA0001377F80F2392E70003C735000D8B9316A9
:103AB0002700370700081307072536971843A38008
:103AC000E700BE85EFF02FD60145B240410182806C
:103AD0009378F70713963800B3071641939627009B
:103AE0009386060CAA969387860033061641931692
:103AF0002600AA9603C6860C136606F82384C60C15
:103B000049BF411106C693978501E18763C2070249
:103B100093973500B385B740939725009385072683
:103B2000AA95B105EFF06FDA0145B24041018280FC
:103B300093F5F507939735008D8F9395270093851F
:103B4000050CAA95A105F9BF411106C613F8F507A2
:103B500013173800B305074193972500938707266D
:103B6000AA979385C7003307074193172700AA97A1
:103B700023AAC72623ACD72623AE07260347450032
:103B800085476308F700EFF06FEA0145B240410155
:103B90008280931738003388074193172800AA972B
:103BA00023A2C728CDB7411106C613F8F50713178E
:103BB0003800B3050741939725009387070CAA9710
:103BC000938587003307074193172700AA9723A8F7
:103BD000C70C23AAD70C23AC070C03474500854725
:103BE0006308F700EFF06FD30145B24041018280D6
:103BF000931738003388074193172800AA9723A00A
:103C0000C70ECDB7411106C693978501E18763C5FD
:103C1000070293973500B385B740939725009385A6
:103C20000726AA95B10585472381F500EFF06FEAD5
:103C30000145B2404101828093F5F5079397350025
:103C40008D8F939527009385050CAA95A105E1BF5B
:103C5000411106C693978501E18763C407029397D4
:103C60003500B385B7409397250093850726AA951D
:103C7000B10523810500EFF08FE90145B240410114
:103C8000828093F5F507939735008D8F93952700E4
:103C90009385050CAA95A105E9BF411106C6EFF071
:103CA0002FB7B2404101828093973500B385B7406A
:103CB000939725003E950355C5278280411106C67E
:103CC000EFF06FB40D45EF001035B2404101828036
:103CD000411106C6EFF06FB20D45EF00D033B24090
:103CE00041018280411106C622C426C22A842328AB
:103CF000C542930485002E86A685EFE05FEE2686FA
:103D000008404C40EFE0BFFF2285D9372285EFF015
:103D10000F992285653785472303F40CB24022446E
:103D2000924441018280054582808327454183C7B3
:103D300007002310F6000325454182808327854133
:103D400083C727002310F60003258541828083273F
:103D5000C54183C727002310F6000325C541828093
:103D6000832705428A05AE978843834705002310C1
:103D7000F600828003C7450083C75500A207D98F8C
:103D800013F6F70F03C705000D8B85466305D708AB
:103D900093168701E18691C689466307D70A0545D0
:103DA00082808347650C93F7F70F0947638BE70021
:103DB0008347650C93F7F70F0D476384E7000545CC
:103DC00082808347054195CFB707002005472386AA
:103DD000E768834725419DCBB70700209387C768D5
:103DE00003C70700136727002380E700B7070020F9
:103DF0009387C7682328F50C8947232EF50C0145C6
:103E00008280B707002023860768E1B7B707002044
:103E100023860768E1BF8347650C93F7F70F0D47CB
:103E20006384E70005458280854763F4C700054544
:103E30008280B70700209387C7682328F50C89473D
:103E4000232EF50C014582800347650C1377F70F8D
:103E50008D466304D70005458280E207E18763CA87
:103E60000702931736003386C74093172600AA9798
:103E700003C7E726B70700202386E768B7070020B7
:103E80009387C7682328F50C8947232EF50C014535
:103E900082801376F607931736003386C740931750
:103EA0002600AA9703C7A70CB70700202386E76858
:103EB000F1B7411106C622C426C2AA842E8483C744
:103EC00005008D8B85C305476386E70C03A7C40DEA
:103ED00065CB8346640083477400A207D58FE1E376
:103EE0000545C5A083C7250083C53500A205DD8D26
:103EF00093D7850093F5F50F0947638EE704637E3A
:103F0000F7000D476387E7063D47E391E7FC13069B
:103F1000C50D353D23A8A40C55BF0547E398E7FA26
:103F2000FD178A073707000813074729BA979C43EC
:103F30001306C50D829723A8A40C0347640083478A
:103F40007400A207D98F13070004E391E7F8A14793
:103F500023AEF40CA5BFFD178A0737070008130727
:103F60004729BA979C431306C50D829723A8A40C32
:103F7000B1BF1547E36CB7F4FD178A073707000890
:103F800013074729BA979C431306C50D829723A8A8
:103F9000A40C2DBF83270543DC4782971DA0637DBA
:103FA000F70083D7C40C636BF7003377F70219E788
:103FB0008547A386F44219A023AEF40C014511A055
:103FC0000545B240224492444101828001458280ED
:103FD0008347650C93F7F70F09476387E7000D47A1
:103FE0006382E702054582808347450C99C30545F6
:103FF00082809307450C2328F50C8547232EF50C6A
:10400000014582808347450C99E3054582809307EB
:10401000450C2328F50C8547232EF50C014582809D
:1040200083C52500B7070020A384B768854763F4DC
:10403000B70005458280411106C622C42A84834701
:10404000650C93F7F70F0947638AE7000D4763870D
:10405000E7020545B24022444101828091CD832789
:104060000543DC438297B707002083C79768230284
:10407000F40C8D472303F40C0145E9BF85E1832748
:1040800005439C478297B707002083C797682302A0
:10409000F40C89472303F40C01456DBF8347450C9D
:1040A000E38CF5FE832705439C478297B7070020E2
:1040B00083C597682302B40C83270443DC4322851D
:1040C0008297D9BF8347650C93F7F70F0D47638439
:1040D000E7000545828003C74500854763F4E70094
:1040E000054582808327054385072328F50C8547EE
:1040F000232EF50C014582808347650C93F7F70F5B
:104100000D476384E7000545828003C74500854766
:1041100063F4E7000545828003C725008327054334
:10412000A380E700014582800145828003C74500E6
:1041300083C75500A207D98FB9EB03C7650083C7B2
:104140007500A207D98FB1E783C5250093F5F50760
:10415000A302B50C8347650C93F7F70F0D476394E3
:10416000E70005458280411106C622C42A843536FF
:104170008347540C89CB89472303F40C0145B24093
:1041800022444101828085472303F40CC5BF0545C5
:1041900082800545828083C705008D8B91C70947C2
:1041A0006383E704054582808347650C93F7F70F27
:1041B0000947638BE7008347650C93F7F70F0D47BB
:1041C0006384E7000545828003C7250083C7350067
:1041D000A207D98F05476384E700014582808547A0
:1041E0002309F540DDBF83C645008347650C93F77F
:1041F000F70F0D476384E7000545828003C725005C
:1042000083C73500A207D98F91E789C693070008B5
:104210006394F60001458280411106C6B685DD3201
:104220000145B2404101828083C705008D8B91C753
:1042300009476383E704054582808347650C93F74C
:10424000F70F0947638BE7008347650C93F7F70F78
:104250000D476384E7000545828003C7250083C7B7
:104260003500A207D98F05476384E70005458280A2
:10427000230905400145828083C645008347650CBC
:1042800093F7F70F0D476384E7000545828003C766
:10429000250083C73500A207D98F91E789C6930708
:1042A00000086394F60001458280411106C622C4CD
:1042B00026C22E84AA84B685EFF09F9983A7044373
:1042C000DC47A285268582970145B240224492446C
:1042D00041018280411106C683C71500139727004C
:1042E000B707000893870726BA979C438297B24086
:1042F000410182808347650C93F7F70F0D47638474
:10430000E7000545828003C74500854763F4E70061
:1043100005458280411106C683270543DC47829705
:10432000B2404101828001458280411106C622C40B
:104330002A8493050008EFF0FF8C81452285EFF079
:104340007F8C2285EFF00F86B240224441018280AB
:10435000411106C622C42A848356C50D0326050DC5
:104360008145EFF05F840327C40D8357C40C63FAC3
:10437000E70085472306F4420145B240224441014B
:10438000828089472306F442C5BF411106C622C474
:104390002A8483560528032645278145EFF0CFFA66
:1043A000032704288357042763FAE7008D47230671
:1043B000F4420145B24022444101828091472306E4
:1043C000F442C5BF411106C622C42A84954723067C
:1043D000F542814601468145EFF0EFFC2285EFE092
:1043E0007FFC0145B240224441018280411106C652
:1043F00022C42A8499472306F54281460146814515
:10440000EFF08FF42285EFE0FFF90145B24022443E
:1044100041018280011106CE22CC2A8483274542A5
:104420003EC4032785423AC693F7070613070002E6
:10443000638CE70213070004638BE70289CB2C002F
:104440002285E5350145F2406244056182802C00F9
:10445000513575F58357E10091CF8307810063CE15
:10446000070022851D37F9BF2C006935DDB72C0008
:104470005D3DC5B72285B937F1B72285D13DD9B7A2
:10448000797106D622D40018232EA4FCAE87A30D82
:10449000F4FC8347B4FDD1E38327C4FD9387C7268B
:1044A0002326F4FE8327C4FD83C7C7420D476386D6
:1044B000E70011476383E70259A88327C4FEDC4B5A
:1044C0000327C4FE035747003387E7408327C4FE12
:1044D000D8CB0325C4FD553D9DA88327C4FD83C7C4
:1044E000670C13F7F70F8D476311F7028327C4FD9D
:1044F00083A70743DC4B91CB8327C4FD83A70743E6
:10450000DC4B81450325C4FD82978327C4FE23AA83
:1045100007000325C4FD7D351DA88327C4FD83A79F
:104520000743DC4B8DC78327C4FD83C7670C13F794
:10453000F70F8D47631DF7008327C4FD83A707434B
:10454000D84B8347B4FDBE850325C4FD0297814740
:104550003E85B250225445618280797106D622D4BC
:104560000018232EA4FCAE87A30DF4FC8347B4FDF2
:10457000DDE38327C4FD9387870C2326F4FE83277E
:10458000C4FD83C7C74205476386E70009476383C5
:10459000E70265A88327C4FEDC4B0327C4FE03574C
:1045A00047003387E7408327C4FED8CB0325C4FDEB
:1045B000453361A88327C4FD83C7D74289CF81468D
:1045C000014681450325C4FDEFF0EFDD8327C4FDDF
:1045D000A38607429DA88327C4FD83C7670C13F7F2
:1045E000F70F8D476311F7028327C4FD83A70743A5
:1045F0009C4B91CB8327C4FD83A707439C4B8145EC
:104600000325C4FD82978327C4FE23AA0700032540
:10461000C4FDE93B1DA88327C4FD83C7670C13F7BE
:10462000F70F8D476313F7028327C4FD83A7074362
:104630009C4B81CF8327C4FD83A70743984B8347B7
:10464000B4FDBE850325C4FD029781473E85B25067
:10465000225445618280011106CE22CC2A841305A2
:104660001070EFE00F893705004013050540EFE0BB
:10467000AFA389476305F40685476305F406B717BA
:10468000002083A7C76A2310F10023110100231221
:10469000010023160100230701008A85370400402A
:1046A00013050440EFE08FAC13050440EFE0AFB812
:1046B000854513050440EFE02FBA854513050440F6
:1046C000EFE0EFBA814513050440EFE04FB7130563
:1046D0000440EFE02FB5F240624405618280AD47AF
:1046E0003EC471BF8D679387F7ED3EC449BF41114A
:1046F00006C6B707002023A8A7682E85A93FB707DD
:10470000002083A70769E5FF370500401305054032
:10471000EFE0EFB1B24041018280411106C6014590
:10472000EFE02F83B777DC02938707C0630AF502B7
:10473000B7A74A0493870720630CF504B7E7B805C9
:10474000938707806319F502B70700203707C00079
:1047500023AAE768B71700201D4723A6E76A21A808
:10476000B70700203707400023AAE768B7170020E3
:104770000D4723A6E76AB707002003A54769EFD0D6
:104780001FFC1305C050EFD0DFF6B240410182801C
:10479000B707002023AA0768B7170020154723A6EC
:1047A000E76AD1BF411106C601468545130560057C
:1047B000EFE0CFAD1305C071EFD0BFF337050400B4
:1047C000EFE0CFBB0146814537050400EFE0AFAE17
:1047D00037050400EFE08FB901468D451305D0037E
:1047E000EFE0CFAAB24041018280411106C6130515
:1047F0001070EFD01FF00146894513050003EFE06C
:10480000EFA8B24041018280411106C68945C535F5
:10481000B24041018280411106C68545C93DB24082
:1048200041018280411106C68545370500401305C8
:104830000540EFE0EFA201E5B240410182808545ED
:104840003705004013050540EFE06FA2B7070020D1
:1048500083A7076989CBB707002093870769984327
:104860007D1798C3D1BF3705004013050540EFE021
:104870000F9CD9B7411106C63705002013058506E0
:10488000EFE0BFB6B240410182808280411106C68E
:10489000B70700209387870683C7770081EB37052A
:1048A0000400EFE0AFADB24041018280EFD0BFD253
:1048B000B707002003A54769EFD07FE81305C05074
:1048C000EFD03FE33705002013058506EFE05FB02A
:1048D000F9B7411106C6B937B24041018280411192
:1048E00006C622C426C2AA8437040020130404008A
:1048F0009305C403EFF0AF95930554032685EFF0BD
:104900000F95930554022685EFF06F940145B24050
:104910002244924441018280411106C622C42A8465
:1049200093051008EFF0EF9D8D452285EFF06F9D08
:10493000930520082285EFF0CF9C0145B240224428
:1049400041018280411106C681C98D476389F50006
:104950000945B2404101828001220945DDBF05477A
:104960002388E1808D45EFF02FB4B707002023ACFA
:10497000A7680145F9BF85476384F5000945828032
:1049800093F6F507939736003386D7401317260022
:104990002A970326470D958F139727002A97835749
:1049A000C70CB377F60291E311E60547A388E180CF
:1049B00001458280411106C681460146EFF0AF9E57
:1049C0000145B2404101828083C7150013070002F0
:1049D0006388E700130710026385E70201458280C0
:1049E00023A2F180B71700209387076F232AF526AB
:1049F00003C7650083C77500A207D98F2320F52858
:104A0000F1BF138781801443B71700202388D76E26
:104A100013D686009387076FA380C70013D60601BD
:104A20002381C700E182A381D70083464700238208
:104A3000D70083465700A382D7000347670023832C
:104A4000E7002328F50C03C7650083C77500A2079C
:104A5000D98F232EF50C59B703A741809307F00F88
:104A60006307F704B717002003C7076F9387076F23
:104A700083C61700A206558F83C62700C206558F2E
:104A800083C63700E206558F9386818098C203C79C
:104A900047002382E60003C75700A382E60083C7CE
:104AA00067002383F6001307F00F23A2E18001457E
:104AB0008280411106C6B70700209387476A23907A
:104AC000070023910700EFD01FFB0945EFD01FFB24
:104AD000A931213BC139370600201306460485451C
:104AE0003705002013058506EFF0CF9FB240410146
:104AF0008280411106C6B707002083D7476A130793
:104B00009003638BE7066372F7061307F003638273
:104B1000E70413071004639EE706B707002083A588
:104B2000876913858184EF2090502DC923880180E7
:104B300093060004138681848D45370500201305F4
:104B40008506EFF06F80B70700201307F00323926C
:104B5000E76A03C7018185476315F704B70700209B
:104B6000130710042392E76A4DBF85E7B7070020BB
:104B7000130790032392E76AB707002093878706FD
:104B800083C7670C93F7F70F0D47E381E7FA0145F9
:104B900031A0B70700202392076A0D45B2404101BA
:104BA00082800145E5BF411106C622C4B707002037
:104BB0009387476A83D727001307C004638FE702F0
:104BC0006374F7021307F004638CE70413074005CE
:104BD000639BE70803C7118185476303F708014515
:104BE000B240224441018280BDEFB7070020938785
:104BF000476A1307C0042391E700B7070020938793
:104C0000870683C7670C93F7F70F0D476395E70691
:104C1000B70700209387476A1307F0042391E70042
:104C2000370400201304446A13058400EF20105158
:104C300048C021C5A3880180370400201304446ABA
:104C4000835684002A869305100837050020130533
:104C50008506EFE05FF5930740052311F4009DBF43
:104C6000EF20704F75B7B70700209387476A2391ED
:104C700007000D45B5B70145A5B7014595B74111E9
:104C800006C6F32700B8732500B0F32500B8E39AF1
:104C9000B7FE130600068146EF40A03DB240410139
:104CA0008280370500081305C5328280411106C68F
:104CB00022C4938781882390070023810700A38162
:104CC000070013052060EFD0DFA289460946C145E1
:104CD0003714014013050480EFD0DF958945130593
:104CE0000480EFD0DFA0930600080946C1451305F4
:104CF0000480EFD03F949305000813050480EFD0A3
:104D00001F9FB240224441018280411106C683D7D1
:104D10008188130710046386E70813075004638E25
:104D2000E70A99C7239401880D45B240410182806A
:104D30009387818883C7270085CB9387818883C722
:104D4000370091CB938781883797980013070768BE
:104D5000D8C398C735A09387818837F7FA0213071D
:104D60000708D8C398C729A89387818837979800E0
:104D700013070768D8C337E7F5051307071098C767
:104D8000930500083715014013050580EFD0FF9506
:104D9000732700B093878188D8C713071004239026
:104DA000E700732700B093878188D447158FDC43D1
:104DB0006374F700014595BF93050008371501405E
:104DC00013050580EFD0BF92732700B093878188C9
:104DD000D8C7130750042390E700732700B09387C8
:104DE0008188D447158F9C47E37EF7F2014535BF94
:104DF000411106C622C42A8415C1894537150140D0
:104E000013050580EFD07F8E33348000938781882F
:104E100023818700B24022444101828089453715B1
:104E2000014013050580EFD09F8CF9BF3335A000FA
:104E300093878188A381A7008280411106C601CD96
:104E4000930500083715014013050580EFD0FF8951
:104E5000B2404101828093050008371501401305D7
:104E60000580EFD0DF88EDB7411106C622C41305D7
:104E70003060EFD01F8889660546C1453714014070
:104E8000130504C0EFD00FFB85660546C145130529
:104E900004C0EFD02FFAA1660546C145130504C032
:104EA000EFD04FF99166014693058004130504C0C5
:104EB000EFD04FF885460546D145130504C0EFD025
:104EC0006FF7B240224441018280411106C622C4DC
:104ED00089660146814537140140130504C0EFD0AF
:104EE0006FF5856601468145130504C0EFD08FF448
:104EF000A16601468145130504C0EFD0AFF391666A
:104F000001468145130504C0EFD0CFF28546014626
:104F10008145130504C0EFD0EFF1B24022444101B6
:104F20008280411106C619C9854537150140130510
:104F300005C0EFD08FFBB240410182808545371517
:104F40000140130505C0EFD08FFAF5B7F32600B086
:104F5000931715003E9513175500F32700B0958F52
:104F6000E3EDE7FE8280411106C6FD3DB717014023
:104F7000056723A8E7C0B240216723A8E7C00967F7
:104F800023AAE7C04101828089B7B71701400568AD
:104F900023AA07C1216823A807C1732800B0F327FB
:104FA00000B0E30EF8FEB7170140096823A807C157
:104FB00083A787C0F32800B07548F32700B0B387F4
:104FC0001741E37CF8FEB7170140096823AA07C11F
:104FD000056823AA07C1216823A807C1732800B068
:104FE000F32700B0E30EF8FEB7170140096823A8C5
:104FF00007C183A787C0F32800B07548F32700B026
:10500000B3871741E37CF8FEB7170140096823AA6C
:1050100007C18148A1C637180140930E48C1856277
:10502000A16F096E754F23A05E002328F8C173237A
:1050300000B0F32700B0E30EF3FE2328C8C1832796
:1050400088C0732300B0F32700B0B3876740E37CC8
:10505000FFFE23A0CE018508E397D8FC130FF6FFCF
:1050600001486305061E411122C626C437130140BC
:105070008562896E754EA163854F935658008A06E6
:10508000B387D50083A807009377F801B3D8F80059
:1050900093F8180063140F01630B0716232A53C0FB
:1050A00063880812232873C0732400B0F32800B06B
:1050B000E30E14FF2328D3C1832883C093D8E800CC
:1050C00093F81800F32400B0732400B0058CE37D3E
:1050D0008EFE232AD3C1AA96B397FF008042638431
:1050E000080EC18F9CC20508E31906F99308F7FF63
:1050F000014621C7B7170140056E21630965F545D3
:10510000638BC80C23AAC7C123A867C0732800B04B
:10511000F32600B0E30ED8FE23A8A7C083A687C05D
:10512000732800B0F32600B0B3860641E3FCD5FE39
:1051300023AAA7C00506E315E6FCB71701400567DB
:1051400023A8E7C0216723A8E7C0732700B0F3278F
:1051500000B0E30EF7FEB7170140096723A8E7C0C8
:1051600083A787C0F32600B07547F32700B0958F5B
:10517000E37DF7FEB7170140096723AAE7C005677B
:1051800023AAE7C0216723A8E7C0732700B0F3274D
:1051900000B0E30EF7FEB7170140096723A8E7C088
:1051A00083A787C0F32600B07547F32700B0958F1B
:1051B000E37DF7FEB7170140096723AAE7C0324431
:1051C000A2444101828093C7F7FFE18F9CC221BFB7
:1051D000232A73C0D1BD23A8C7C123A867C07328E1
:1051E00000B0F32600B0E30ED8FE23A8A7C083A624
:1051F00087C0732800B0F32600B0B3860641E3FCF5
:10520000D5FE23AAA7C00506E31CE6EE3DB723287A
:1052100053C0638A0802232873C0732400B0F328A4
:1052200000B0E30E14FF2328D3C1832883C093D892
:10523000E80093F81800F32400B0732400B0058C44
:10524000E37D8EFE79B5232A73C0C1BF9308F7FFB3
:10525000014621C7B7170140056E21630965F54571
:105260006380C80C23AAC7C123A867C0732800B0F5
:10527000F32600B0E30ED8FE23A8A7C083A687C0FC
:10528000732800B0F32600B0B3860641E3FCD5FED8
:1052900023AAA7C00506E315E6FCB717014005677A
:1052A00023A8E7C0216723A8E7C0732700B0F3272E
:1052B00000B0E30EF7FEB7170140096723A8E7C067
:1052C00083A787C0F32600B07547F32700B0958FFA
:1052D000E37DF7FEB7170140096723AAE7C005671A
:1052E00023AAE7C0216723A8E7C0732700B0F327EC
:1052F00000B0E30EF7FEB7170140096723A8E7C027
:1053000083A787C0F32600B07547F32700B0958FB9
:10531000E37DF7FEB7170140096723AAE7C0828043
:1053200023A8C7C123A867C0732800B0F32600B024
:10533000E30ED8FE23A8A7C083A687C0732800B0B9
:10534000F32600B0B3860641E3FCD5FE91B7B7174C
:105350000140056723A8E7C0216723A8E7C0F3271A
:1053600000B0732700B0E38EE7FEB717014009676E
:1053700023A8E7C083A787C0F32600B07547F327AB
:1053800000B0958FE37DF7FEB7170140096723AAA8
:10539000E7C0054781466FF05FBFB717014005675B
:1053A00023A8E7C0216723A8E7C0F32700B073272D
:1053B00000B0E38EE7FEB7170140096723A8E7C0F6
:1053C00083A787C0F32600B07547F32700B0958FF9
:1053D000E37DF7FEB7170140096723AAE7C0056719
:1053E00023A8E7C0216723A8E7C0F32700B07327ED
:1053F00000B0E38EE7FEB7170140096723A8E7C0B6
:1054000083A787C0F32600B07547F32700B0958FB8
:10541000E37DF7FEB7170140096723AAE7C01547E8
:1054200081466FF09FB6371701401946930607C1B2
:105430000563A1680965754823A0660023A01601CD
:10544000F32500B0F32700B0E38EF5FE88C2832772
:1054500087C0F32500B0F32700B08D8FE37DF8FE01
:10546000930747C1232AA7C07D1679F6856694C3A2
:10547000A1672328F7C0732700B0F32700B0E30E1D
:10548000F7FEB7170140096723A8E7C083A787C0C5
:10549000F32600B07547F32700B0958FE37DF7FE44
:1054A000B7170140096723AAE7C0828021C53717D3
:1054B00001408146130847C1056E21638965F5489F
:1054C0002320C801232867C0732600B0F32700B04B
:1054D000E30EF6FE2328B7C0832787C0732600B0EB
:1054E000F32700B0918FE3FDF8FE2320B800850676
:1054F000E318D5FC82803705000813050534828047
:1055000005651305C5718280411106C622C42A842F
:105510009387818983D727001307E01E6382E706FC
:10552000637AF7021307201F6387E7081307501FEA
:105530006390E70A9385818913864510D10511454B
:10554000EF10B033854763F7A70C93878189DC4B55
:105550001CC0BDA8D9C71307C01E639BE70693876D
:10556000818913864710AC535D45EF10D0428547C3
:1055700063FCA708938781891307E01E2391E70046
:1055800093858189138645109385C5055945EF108C
:10559000D02E854763FCA70693878189FC4F93F73C
:1055A0000770A1CF9387818913070070F8CF130785
:1055B000201F2391E7009387818913864710EC4FC2
:1055C0005945EF10503D854763F4A704FD571CC0B3
:1055D00093878189239107000D45B2402244410100
:1055E00082809387818937072200B8D32390B7063A
:1055F0001307C01E2391E7009DB793878189130786
:10560000501F2391E7003DB70145C1BF0145F1B7E8
:105610000145E1B70145D1B7411106C622C49387C0
:10562000818983D7270013079020638CE7062E8497
:10563000637EF7021307B0206386E7081307F020A4
:10564000639DE7009387818913864710EC4F594586
:10565000EF107034854763F0A70C938781892391FD
:1056600007000D45B240224441018280C1CB13079F
:105670001020E394E7FE1386818913064610AA855D
:105680001145EF105031854763F1A7089387818951
:1056900037072300B8D32390870613079020239160
:1056A000E7009387818913864710AC535D45EF105F
:1056B000902E854763FDA704938781891307B02047
:1056C0002391E70093858189138645109385C5054D
:1056D0005945EF10901A854763FDA702938781898A
:1056E000FC4F93F70770B5DB938781891307007030
:1056F000F8CF1307F0202391E700A9B7938781899A
:10570000130710202391E700BDB70145A1BF014554
:1057100091BF014581BF0145B1B7411106C622C401
:105720002A849387818983D727001307B025638D47
:10573000E7066377F702130710266381E70C130768
:1057400040266387E70E1307D025638EE70693870D
:105750008189239107000D45B24022444101828096
:10576000C5CF13075025E394E7FE938781891386FD
:1057700047108C4F1545EF101022854763FAA70C90
:105780009387818923A007060947A381E706B853B9
:10579000B70690FFFD16758FB7062000558FB8D35A
:1057A0001307B0252390E70093878189138647105C
:1057B000AC535D45EF10301E854763FDA708130706
:1057C000D025239CE1889385818913864510938594
:1057D000C5055945EF10700A854763FFA7069387F3
:1057E0008189FC4F93F70770A1C3938781891307C1
:1057F0000070F8CF130710262390E7009387818964
:1058000013864710EC4F5945EF10F018854763F7A2
:10581000A704FD571CC025BF938781898CCF130730
:1058200050252390E70091B713074026239CE18879
:105830009385818913864510D1051145EF10F0033A
:10584000854763FFA70093878189DC4B1CC001B7A4
:10585000014519B7014509B70145FDBD0145EDBD3C
:105860000145DDBD411106C622C42A849387818982
:1058700083D727001307F023638DE7066377F702CA
:10588000130750246381E70C130780246388E70E15
:1058900013071024638EE7069387818923910700FD
:1058A0000D45B240224441018280CDCF13079023A1
:1058B000E394E7FE93878189138647108C4F154543
:1058C000EF10700D854763FCA70C9387818923A097
:1058D00007060947A381E706B853B70690FFFD16F0
:1058E000758FB7061000558FB8D31307F023239098
:1058F000E7009387818913864710AC535D45EF100D
:105900009009854763FFA70813071024239CE188AB
:1059100093858189138645109385C5055945EF10F8
:10592000C075854763F1A70893878189FC4F93F77A
:105930000770A9C39387818913070070F8CF1307F5
:1059400050242390E7009387818913864710EC4FFA
:105950005945EF105004854763F9A704FD572310FC
:10596000F4001DBF938781898CCF13079023239068
:10597000E70089B713078024239CE18893858189F8
:1059800013864510D1051145EF10206F854763F050
:10599000A70293878189DC4B2310F400F5BD0145F4
:1059A00009B70145FDBD0145EDBD0145DDBD014521
:1059B000CDBD411106C622C42A849387818983D72D
:1059C000270013073022638AE7066377F70213077D
:1059D0009022638EE70A1307C0226385E70E130740
:1059E0005022638BE70693878189239107000D4539
:1059F000B240224441018280D5CB1307D021E394E9
:105A0000E7FE93878189138647108C4F1545EF1069
:105A10008078854763F9A70C9387818923A00706BF
:105A20000947A381E706B853B70690FFFD16758FA7
:105A3000B8D3130730222390E70093878189138618
:105A40004710AC535D45EF100075854763FFA7080D
:105A500013075022239CE188938581891386451082
:105A60009385C5055945EF104061854763F1A70847
:105A700093878189FC4F93F70770A9C39387818926
:105A800013070070F8CF130790222390E700938745
:105A9000818913864710EC4F5945EF10C06F854739
:105AA00063F9A704FD572300F40035BF938781896C
:105AB0008CCF1307D0212390E700A1B71307C02292
:105AC000239CE1889385818913864510D105114572
:105AD000EF10A05A854763F0A70293878189DC4BBA
:105AE0002300F40009B7014521B7014511B701456D
:105AF00001B70145F5BD0145E5BD411106C622C40A
:105B00009387818983D727001307902A6382E7064A
:105B10002A846377F7021307202B638BE70A1307A6
:105B2000602B6382E70E1307002B6384E7089387DB
:105B30008189239107000D45B240224441018280B2
:105B40006380070E1307702AE393E7FE938781892A
:105B5000138647108C4F1545EF10E063854763F9B6
:105B6000A70C93878189C0CB1307902A2390E70065
:105B70009387818913864710CC4B1145EF10A061A4
:105B8000854763F9A70A9387818923A007060947F8
:105B9000A381E706B853B70690FFFD16758FB706C9
:105BA0002000558FC166558FB8D31307002B239063
:105BB000E7009387818913864710AC535D45EF104A
:105BC000805D854763FAA7061307202B239CE18895
:105BD00093858189138645109385C5055945EF1036
:105BE000C049854763FCA70493878189FC4F93F7DD
:105BF000077095DF9387818913070070F8CF13072B
:105C0000602B2390E7009387818913864710EC4F20
:105C10005945EF1040588547E3EBA7F0014529BFF0
:105C2000938781898CCF1307702A2390E70039BFAF
:105C3000014519B7014509B70145FDBD0145EDBD58
:105C4000411106C622C49387818983D72700130791
:105C5000E0286382E7062A846377F7021307702936
:105C6000638BE70A1307B0296382E70E13075029F5
:105C70006384E70893878189239107000D45B2402B
:105C80002244410182806380070E1307C028E393FA
:105C9000E7FE93878189138647108C4F1545EF10D7
:105CA000804F854763F9A70C93878189C0CB130781
:105CB000E0282390E7009387818913864710CC4B17
:105CC0001145EF10404D854763F9A70A93878189F5
:105CD00023A007060947A381E706B853B70690FF3C
:105CE000FD16758FB7061000558FC166558FB8D356
:105CF000130750292390E700938781891386471063
:105D0000AC535D45EF102049854763FAA70613079A
:105D10007029239CE188938581891386451093859A
:105D2000C5055945EF106035854763FCA704938787
:105D30008189FC4F93F7077095DF9387818913075B
:105D40000070F8CF1307B0292390E700938781896B
:105D500013864710EC4F5945EF10E0438547E3EBBE
:105D6000A7F0014529BF938781898CCF1307C028ED
:105D70002390E70039BF014519B7014509B701452F
:105D8000FDBD0145EDBD411106C622C49387818941
:105D900083D72700130730276382E7062A846377B7
:105DA000F7021307C0276388E70A13070028638FE9
:105DB000E70C1307A0276381E70893878189239164
:105DC00007000D45B240224441018280638D070CDB
:105DD00013071027E393E7FE938781891386471003
:105DE0008C4F1545EF10203B854763F6A70C938732
:105DF0008189C0CB130730272390E70093878189DF
:105E000013864710CC4B1145EF10E038854763F6F9
:105E1000A70A9387818923A007060947A381E7067C
:105E2000B853B70690FFFD16758FC166558FB8D36E
:105E30001307A0272390E7009387818913864710D3
:105E4000AC535D45EF102035854763FAA70613076D
:105E5000C027239CE188938581891386451093850B
:105E6000C5055945EF106021854763FCA70493875A
:105E70008189FC4F93F70770A9D393878189130712
:105E80000070F8CF130700282390E70093878189DB
:105E900013864710EC4F5945EF10E02F8547E3EE8E
:105EA000A7F0014505B7938781898CCF1307102789
:105EB0002390E70015B7014531B7014521B70145EA
:105EC00011B7014501B7411106C693878189239017
:105ED00007002391070023A407109387818983A7D4
:105EE00087100D476361F7021387818913961700A6
:105EF0003E9693162600BA96154623A2C61285072B
:105F00002324F710D9BFEF104015B2404101828021
:105F1000411106C622C42A8483D78189130730061B
:105F20006384E7086378F7041307B0066387E70A1A
:105F3000130710076397E71093858189138645102F
:105F4000938545044145EF104013854763F8A7103A
:105F50009387818983A74710639D070C9387818965
:105F6000F8438547630DF70C8D471CC0239C0188BF
:105F70000945D9A8C1CB1307D0056394E70C138555
:105F8000818913050511EF009066854763F2A70C20
:105F90009387818983A70711FD1775576369F706F2
:105FA00013073006239CE188138581891305451169
:105FB000EF007073854763FFA7089387818983A7E4
:105FC0004711BD8B0547639AE7049387818905478D
:105FD000F8C31307B0062390E700938781891386DF
:105FE0004710EC434145EF10001B854763F6A706B9
:105FF0009387818983A747109DE713071007239C88
:10600000E1881DBF1307D005239CE1888DBF85471C
:106010001CC0239C0188094505A889471CC0239CF6
:106020000188094515A08D471CC0239C018809459E
:1060300021A88D471CC0239C0188094531A023203D
:106040000400239C01880D45B24022444101828016
:106050000145DDBF0145CDBF0145FDB70145EDB7A8
:1060600083D7818989CB1307C008638EE700239CFF
:1060700001880D4582809387818923A20704130735
:10608000C0082390E700411106C6938781891386D3
:106090004710EC434145EF100010854763F8A70017
:1060A000239C01880D45B240410182800145E5BF36
:1060B000411106C6EF00907BB24041018280938778
:1060C000818903A507118280411106C622C42A8452
:1060D00083D781891307800A638AE7021307A00A1E
:1060E0006386E70681CB239C01880D45B24022449C
:1060F000410182802320050093878189054723A4DD
:10610000E71015A81307800A239CE18893878189EB
:1061100083A78710139527008565BE952295EFF01C
:10612000AFBE854763FFA7029387818903A78710C6
:10613000050723A4E7109387818903A78710FD47EC
:10614000E3F2E7FC1307A00A239CE1889305107B88
:1061500013050408EFF04FBB8547E3E6A7F80145B8
:1061600071B7014561B7411106C622C42A8483D79D
:1061700081891307500B6388E7021307700B63854F
:10618000E70681CB239C01880D45B24022444101A2
:10619000828093878189054723A4E7101DA81307F0
:1061A000500B239CE1889387818903A7871093175D
:1061B0002700A2978565BA958843EFF0EFC585471C
:1061C00063FFA7029387818903A78710050723A48C
:1061D000E7109387818903A78710FD47E3F1E7FC68
:1061E0001307700B239CE1889305107B032504089B
:1061F000EFF08FC28547E3E7A7F8014579B701457E
:1062000069B7411106C622C42A8483D7818913073E
:10621000400C6389E7086375F7021307800C6386F7
:10622000E70A1307A00C6388E70C1307600C638C64
:10623000E704239C01880D45B2402244410182803D
:1062400099CF1307200CE396E7FE8567BE9522855C
:10625000EFF08FAB8547E3EEA7FC0145F1BFFD47AB
:1062600063C7B7001307200C239CE188F9BF93078D
:1062700000026385F5029307000463CFB70213079A
:10628000600C239CE1888567FD17BE952285EFF0A1
:10629000AFA78547E3EFA7F8014579BF1307400C87
:1062A000239CE1889305107B2285EFF0EFA58547BD
:1062B000E3E1A7F8014549B785679387070463C001
:1062C000B7021307800C239CE1889385F5FB228598
:1062D000EFF08FA38547E3EEA7F40145B1BF8567D3
:1062E000938717046385F500FD571CC199B7130701
:1062F000A00C239CE1889305007B138581891305FD
:10630000C510EFF06FA0854763F9A70093878189D7
:1063100083A7C7108D8B1CC029BF014531BF411118
:1063200006C683D781891307B00D6389E7086373B5
:10633000F7021307D00D6385E7061307F00D639787
:10634000E7029385F5FBEFF02FAD854763E0A702E9
:10635000014505A095C31307900D6399E700856774
:10636000BE95EFF06FAB854763FDA706239C0188C0
:106370000D45B24041018280FD4763C7B700130756
:10638000900D239CE188E1BF930700026384F5022E
:106390009307000463CDB7021307D00D239CE18857
:1063A0008567FD17BE95EFF02FA78547E3E0A7FCB3
:1063B0000145C1B71307B00D239CE1889305107BFD
:1063C000EFF08FA58547E3E3A7FA01455DB7856741
:1063D00093870704E3CCB7F81307F00D239CE188FB
:1063E0008DB7014579B7411106C622C426C24AC0FD
:1063F0002A84AE84328983D781891307E00E638DA6
:10640000E7066378F7041307200F638BE70C130785
:10641000600F639CE7089387818903A58710B30504
:1064200095002295EFF0EFD8854763FEA70E93877E
:10643000818903A78710050723A4E7109387818923
:1064400083A7871063F327071307600F239CE18856
:10645000D9B7A1EF93773500B5E393F73500B9EFDE
:1064600093773600A1EF9387818923A4071005A8AD
:106470001307E00E239CE1889387818903A5871089
:10648000B30595002295EFF04FA9854763F9A7085A
:106490009387818903A78710110723A4E7109387A7
:1064A000818983A78710E3E527FD239C01880D459B
:1064B000B240224492440249410182809377140001
:1064C000B1EB93F71400B9E793771900A1E793872D
:1064D000818923A4071005A81307200F239CE188B6
:1064E0009387818903A58710B30595002295EFF066
:1064F0006FB7854763F7A7029387818903A7871042
:10650000090723A4E7109387818983A78710E3E510
:1065100027FD61BF9387818923A4071005B7014533
:1065200041BF014571B7014561B7411106C622C49B
:1065300026C24AC02A842E89B28483D78189130750
:1065400040106380E708637AF70413078010638BB9
:10655000E70C1307C0106393E7129387818983A523
:106560008710B307B400CA9503C50700EFF0BF81D9
:10657000854763F2A7129387818903A787100507D0
:1065800023A4E7109387818983A7871063F5970673
:106590001307C010239CE188C9B76391070E937756
:1065A0003500B9EF93F73500A1EF93773600A9EBEB
:1065B0009387818923A407100DA813074010239CFB
:1065C000E1889387818983A58710B307B400CA95B2
:1065D0008843EFF08FD2854763FBA70A93878189B1
:1065E00003A78710110723A4E7109387818983A746
:1065F0008710E3E497FC9387818923A407108DA873
:1066000093771400A1EF93771900A9EB93F7140087
:10661000B1E79387818923A4071015A81307801079
:10662000239CE1889387818983A58710B307B400F1
:10663000CA9503D50700EFF0AFE0854763FBA704D9
:106640009387818903A78710090723A4E7109387FD
:10665000818983A78710E3E397FC71BF93878189C2
:1066600023A4071005B78507138781892324F71012
:106670009387818983A78710E3E797FE239C01888E
:106680000D45B240224492440249410182800145B5
:10669000CDBF0145FDB70145EDB7411106C683D712
:1066A00081891307C0126383E708637BF70213072E
:1066B000F012638CE70E1307C013639DE700938706
:1066C000818913864710EC434145EF00D02C854764
:1066D00063FDA710239C01880D45B24041018280D3
:1066E000CDC713071012E397E7FE938781891386BE
:1066F0004710EC434145EF00102A854763F1A70E90
:106700000145EFE01F8261651305056AEFE01F8414
:106710000545EFE01F819387818937070080136764
:106720009700F8C31307C0122390E700938781896D
:1067300013864710EC434145EF00F025854763F28F
:10674000A70A9387818923A407109387818903A7C8
:1067500087109307300663F6E7049387818937072C
:10676000008013675700F8C3BC471397C7006359ED
:10677000070093878189F843B7060010558FF8C347
:106780001307C013239CE1881DBF938781893707B6
:1067900000801367B700F8C3130710122390E700B7
:1067A000A9B71307F012239CE1889385818913868A
:1067B0004510938585044545EF00300C854763F40B
:1067C000A70293878189BC4793F70720D9F793875E
:1067D000818903A78710050723A4E710BDB70145EA
:1067E000EDBD0145DDBD0145CDBD0145FDB5411105
:1067F00006C683D78189130760146381E7021307F4
:10680000A0146388E70499C7239C01880D45B24012
:106810004101828013076014239CE188938581895C
:1068200013864510938545044145EF0010058547C3
:1068300063FEA70293878189F843B70600C0FD165F
:10684000758FB7060080558FF8C31307A0142390E7
:10685000E7009387818913864710EC434145EF0099
:1068600090138547E3E2A7FA014555B7014545B7BF
:1068700083D7818989CB13074015638AE700239C5E
:1068800001880D45828013074015239CE188411142
:1068900006C622C42A849385818913864510938570
:1068A00085044545EF00607D854763F4A702938723
:1068B0008189BC4793F7072091CB85471CC0239C57
:1068C00001880D45B240224441018280232004000A
:1068D000FDB70145C5BF411106C683D7818913079E
:1068E00060166388E706637BF702130780166381EF
:1068F000E7081307B016639DE70093878189138625
:106900004710EC434145EF001009854763FAA70A99
:10691000239C01880D45B24041018280D9C71307ED
:106920004016E397E7FE9305007B138581891305E5
:10693000C510EFE07FBD854763FEA7069387818979
:1069400003A7C7106D9B23A6E710130760162390BB
:10695000E7009305007B9387818903A5C710EFE0CB
:10696000BFCB854763FAA70413078016239CE188F1
:106970009385818913864510938545044145EF0031
:10698000C06F854763FCA70293878189F843B706E8
:10699000008093C6F6FF758FB7060040558FF8C389
:1069A0001307B0162390E70089BF13074016239CF6
:1069B000E18895BF014585B70145B1BF0145A1BF3C
:1069C000014591BF411106C683D78189130770170E
:1069D0006389E706637BF702130790176382E70872
:1069E0001307C017639DE7009387818913864710BB
:1069F000EC434145EF00207A854763FAA70A239CC0
:106A000001880D45B24041018280D9C71307501754
:106A1000E397E7FE9305007B138581891305C51075
:106A2000EFE09FAE854763FEA7069387818903A7A2
:106A3000C7101367470023A6E710130770172390AA
:106A4000E7009305007B9387818903A5C710EFE0DA
:106A5000BFBC854763F9A70413079017239CE188FF
:106A600093858189138645109385450441453125D9
:106A7000854763FCA70293878189F843B7060080A6
:106A800093C6F6FF758FB7060040558FF8C31307FE
:106A9000C0172390E70089BF13075017239CE18894
:106AA00095BF014585B70145B1BF0145A1BF01456E
:106AB00091BF411106C622C426C22A84B68483D758
:106AC00081891307E018638CE7046376F7021307E4
:106AD000601B6385E7141307701B6387E7161307B2
:106AE000501B638EE710239C01880D45B240224461
:106AF000924441018280D9C31307D018E395E7FE81
:106B00009305007A9387818903A58711EFE0DFB0B1
:106B1000854763F8A7181307E018239CE1889305BD
:106B2000107A138581891305C511EFE0FF9D854714
:106B300063FBA716138781898327C711B70600084F
:106B4000D58FC576FD16F58F8566D58F93E78704BB
:106B5000232EF7108947630EF41063F387088D47DF
:106B60006302F41291476318F4089387818903A79D
:106B7000C7111367370023AEE710B5A89387818943
:106B800023A407109387818983A787100D47636823
:106B9000F70C139717003E979316270013878189E8
:106BA00036978326471215476388E60085071387C3
:106BB00081892324F710F9B79386818913971700E9
:106BC0003E970A073697232287122324B7122326DB
:106BD000C71223ACF6109307D0182390F6000DB718
:106BE0008547631AF4009387818903A7C711136748
:106BF000470023AEE7101307501B239CE188930541
:106C0000107A9387818903A5C711EFE0FFA085471C
:106C100063FDA7081307601B239CE1889387818984
:106C200083A687111397160036970A07BA9793051C
:106C3000207A03A58712EFE03F9E854763F9A706F8
:106C40001307701B239CE1889305107A13858189B3
:106C500013050512EFE05F8B854763FCA70493875C
:106C6000818903A7871091476307F70223A00400D7
:106C70009DBD9387818903A7C7111367270023AEA2
:106C8000E71095BF9387818903A7C7111367170082
:106C900023AEE7108DB7B9479CC0239C01880945F6
:106CA000B1B50145A1B5014591B5014581B5014594
:106CB00035BD014525BD411106C622C4368483D7A2
:106CC00081891307801D6384E7081307901D638F74
:106CD000E70881CB239C01880D45B2402244410145
:106CE00082809387818923A4071031A085071387A9
:106CF00081892324F7109387818983A787100D4703
:106D00006360F70493961700BE96139826001387C6
:106D10008189429703274712E31AA7FC13878189C9
:106D2000429703278712E313B7FC138781894297A1
:106D30000327C712E31CC7FA13878189232CF71096
:106D400011476386E7061307801D239CE18893059E
:106D5000007A9387818903A58711EFE0FF8B854730
:106D600063FDA7041307901D239CE1889305107A07
:106D70000145EFE07F8A854763F3A7049387818904
:106D800003A6871013171600B305C70093962500B6
:106D9000BE96954523A2B61223A4061232979316E7
:106DA0002700B69723A607122320040025B7B9476A
:106DB0001CC0239C018809450DB7014539BF014519
:106DC00029BF411106C69387C19E23900700238ADD
:106DD0000700EFE04F99EFE00FE5B24041018280FC
:106DE000411106C6EFE04F9AB2404101828083D73D
:106DF000C19EB9EF411106C622C426C2AA84938758
:106E0000C19E03C7470185476318F7021384C19EDB
:106E10002322040013060002930544001305C40056
:106E2000EFE0EFD25C449CC02396019E0D45B2403A
:106E300022449244410182801385C19E5CC1230A91
:106E4000F5001546930545003105EFE00FD57DBFF0
:106E50002396019E0D45828083D7C19EA5E34111F3
:106E600006C622C49387C19E03C74701C147631862
:106E7000F7021384C19EC1675CC01306000293052C
:106E800044001305C400EFE08FCC0345540105E531
:106E90002396019E0D45B240224441018280138514
:106EA000C19E5CC1230AF5001546930545003105D6
:106EB000EFE0AFCE7DBFEFE06FDFD9BF2396019E3D
:106EC0000D45828083D7C19E89C72396019E0D45BB
:106ED0008280411106C6EFE06FDD2396019E0D45CD
:106EE000B2404101828083D7C19EBDEF411106C6E9
:106EF00022C426C2AA849387C19E03C74701C14703
:106F00006318F7041384C19E2322040013060002B1
:106F1000930544001305C400EFE06FC35C449CC0BC
:106F2000918393F7F7032301F4009C40B1839D8B79
:106F3000A30AF40091C7FD171387C19EA30AF700A7
:106F40002396019E0D45B240224492444101828025
:106F50001385C19E5CC1230AF500154693054500C3
:106F60003105EFE08FC379BF2396019E0D458280E6
:106F700083D7C19E639F070C011106CE22CC26CA7F
:106F80004AC84EC63289AE84AA899387C19E03C778
:106F900027008547B397E700FD1763ECA70091CD65
:106FA00009C618428D4763FEE7000545EFD0FFE8AC
:106FB00001A00545EFD07FE801A00545EFD0FFE730
:106FC00001A09387C19E03C74701C5476314F70615
:106FD0009C408A07032709000D8BD98F1384C19E1B
:106FE0005CC09C40F9838A09B3E737011CC403469F
:106FF000240013062602930544001305C400EFE0A5
:107000000FB50345540139E11387C19E5C478D8B51
:107010002320F9005C478983184B7A07D98F9CC0DD
:107020002396019E0D45F2406244D2444249B24942
:10703000056182801385C19E5CC1230AF500154657
:10704000930545003105EFE04FB559B7EFE00FC6A6
:1070500065BF2396019E0D458280411106C623928D
:1070600001A0EFF01FD6B24041018280411106C657
:10707000EFF01FD7B24041018280411106C622C401
:1070800026C2AE84328483D741A01307F003638104
:10709000E708637CF702130720046384E70C1307F7
:1070A000A004639CE700EFF03FDB854763F3A70E86
:1070B00009C4938741A0DC471CC0239201A00D4561
:1070C000B2402244924441018280ADCF1307900325
:1070D000E395E7FE938541A01386C500A105EFF077
:1070E0003FE9854763F1A70A938741A023A20700E0
:1070F000938741A0D843954763EDE702938741A06A
:1071000023A4070023A607001307F0032390E7003A
:10711000938541A01386C500A1050145EFF05FE509
:10712000854763F4A706938741A0D8478D47630638
:10713000F702938741A0DC47B1C31307A004239251
:10714000E1A095B7938741A023A407000547D8C7BE
:10715000130790032390E700B5BF13072004239281
:10716000E1A013050002EFF0FFD5854763F1A70208
:10717000938741A0D8430507D8C39DBF938741A0FB
:107180009C479CC035B7014525BF014515BF01454A
:1071900005BF014535B7411106C622C4328483D7E5
:1071A00041A01307E0056387E704637BF702130739
:1071B00030066385E70613077006639CE700EFF06F
:1071C000BFC9854763F4A70809C4938741A0DC477A
:1071D0001CC0239201A00D45B2402244410182808F
:1071E000EDFB938741A08CC70947D8C71307E0057B
:1071F0002390E700938541A01386C500A105EFF019
:107200003FD7854763F0A704938741A023A40700D5
:1072100023A60700130730062390E700938541A0BB
:107220001386C500A1050145EFF09FD4854763FD96
:10723000A700938741A0DC47C1DB130770062392A8
:10724000E1A0B5BF014549BF014579B7014569B71F
:10725000411106C6EFE03FC7239A01A0B2404101A9
:10726000828083D741A189CB13076004638AE7003A
:10727000239A01A00D45828013076004239AE1A0A0
:10728000411106C622C42A84EFE09FC8854763F9EE
:10729000A7021C4081CB239A01A00D45B240224495
:1072A00041018280EFE0BFE1B75700109387D763B9
:1072B000E303F5FE89471CC0239A01A00945F9BFE5
:1072C0000145E9BF83D741A189CB13077005638AC4
:1072D000E700239A01A00D45828013077005239AC9
:1072E000E1A0411106C6EFE0BFD7854763F8A700CC
:1072F000239A01A00D45B240410182800145E5BFBE
:10730000411106C6EFE0DFDAB2404101828041114F
:1073100006C622C426C24AC0AA842E89328483D7D4
:1073200041A11307E0066382E7186378F7061307A5
:107330009007638AE70A6374F7081307B007638A44
:10734000E70C130720086393E7061146B7250240B0
:10735000B105138541A13105EFF0EF88854763FD45
:10736000A71C138541A11105EF10F03E11E593878D
:1073700041A1DC47858BF9E3938741A1DC4713F7F3
:10738000170063100718C18B63930718938741A1F7
:10739000984B1307074098CB81A213079006638F81
:1073A000E70A1307B0066382E70ED1CF239A01A044
:1073B0000D45B240224492440249410182801307A4
:1073C0008007E395E7FE1146B7250240C105138506
:1073D00041A13105EFF06F95854763F9A7141307B5
:1073E0009007239AE1A01146B7250240D1051385E5
:1073F00041A14105EFF06F93854763FBA712938787
:1074000041A1D84713670704D8C71307B0072390D3
:10741000E7001146B7250240C105138541A131059A
:10742000EFF0AF90854763F7A710B7250900938564
:10743000057C138541A11105EF107030130720085A
:10744000239AE1A019B7938741A13707674513072E
:107450003712D8C7130790062390E7001146B725C7
:1074600002409105138541A13105EFF00F8C85474E
:1074700063F8A70A938741A13797EFCD1307B79A0F
:10748000D8C71307B0062390E7001146B72502407E
:107490009105138541A13105EFF02F89854763F3ED
:1074A000A7081307E006239AE1A01146B72502407A
:1074B000C105138541A13105EFE0FFF2854763F572
:1074C000A706938741A1DC4793F707088DE79387C9
:1074D00041A184CBCA94C4CB938741A1984BDC4B88
:1074E000637DF702938741A10947D8C71307800737
:1074F0002390E700C9BD85471CC0239A01A0094518
:107500004DBD89471CC0239A01A009455DB58D4733
:107510001CC0239A01A0094569BD2320040079B548
:10752000014541BD014571B5014561B5014551B503
:10753000014541B50145B5BD0145A5BD011106CEC9
:1075400022CC26CA4AC84EC62E843289B68483D736
:1075500041A11307700A638FE70CAA896379F706C4
:107560001307900A6386E70E1307C00A6397E704C0
:107570001146B7250240B105138541A13105EFE061
:107580009FE6854763F9A710938741A1DC4713F76E
:1075900017006310070E918B6393070E938741A129
:1075A000984B110798CB984F110798CF938741A11B
:1075B0009C4F63EF870423A00400239A01A00D458C
:1075C000F2406244D2444249B2490561828085CB8F
:1075D0001307D009E393E7FE1146B7250240C10522
:1075E000138541A13105EFE05FF4854763FFA708EC
:1075F000938741A123A8370123AC070045BF938798
:1076000041A10547D8C71307D0092390E700E9B780
:10761000938941A19305802513854900EF1030120D
:1076200083A78901CA979C4323A6F9009307700A90
:107630002390F900138541A111460C493105EFE073
:10764000DFEE854763F5A7041307900A239AE1A0AC
:10765000138541A11105EF10101005CD938741A1AD
:1076600083C70701E39C07F21307C00A239AE1A02E
:1076700001B789479CC0239A01A0094591B78D475E
:107680009CC0239A01A0094525BF014515BF0145AE
:1076900005BF014535B7014525B783D741A189CB42
:1076A0001307500C638FE700239A01A00D458280D9
:1076B000938741A113070008D8C71307500C2390E4
:1076C000E700411106C61146B7250240C1051385E2
:1076D00041A13105EFE07FE5854763F8A700239AD4
:1076E00001A00D45B240410182800145E5BF37252B
:1076F0000008130505A68280372500081305C5A6D6
:1077000082801305B00F82808147014763F9B7007B
:10771000B306F50083C6060036978507C5BF137507
:10772000F70F8280938701A323A007007D5798C796
:10773000D8C723A80700238A0700938701E50547D8
:107740002380E700A380070023A20700828015A002
:10775000138701A33E9783465701130740026396A0
:10776000E602138701A31CC70DA08507138701A399
:107770001CCB138701A31C4B184363FBE702138741
:1077800001A314477D57E385E6FC138701A3544703
:107790007D57E39CE6FC138701A33E978346570180
:1077A00013073002E393E6FC138701A35CC775BFA0
:1077B000938701A39C4763C70700938601A3D44620
:1077C0006345D0028547631EF702938701A303C771
:1077D00057018D476319F702138501A38547230AD3
:1077E000F50085475CC155058280138501A30547D7
:1077F000230AE5009D8EFD1654C1C5073E9515056B
:1078000082800145828001458280938701A3C8431D
:107810008280938701A3238A070023A0070023A265
:1078200007007D5798C7D8C723A807008280938791
:1078300001A383C74701B9E383A601A313078040CF
:10784000158F6374B7003E858280411106C622C43D
:1078500026C22E84AA85938401A3C106A6962286F9
:1078600013855600EF10703A8C40A2958CC0854766
:107870003E85B24022449244410182808147E1B773
:1078800083C701E589C7138501E539058280014574
:107890008280938701E523800700C8C393F7150012
:1078A0008DC7938701E513074002A386E70083C7CE
:1078B000170099EF938701E51307B0022386E700CD
:1078C00023A4070013072500D8C3898991E9828082
:1078D000938701E5054798C713071500D8C3F5B787
:1078E000411106C622C426C24AC0AA85138401E5F6
:1078F000032944000444B3079900A29713073002F8
:107900002386E7000509232224011305E400EFF094
:10791000BFDFCA94A294AA8637260008130686B64B
:107920008D451385C400EF1030445C4089075CC06E
:10793000B2402244924402494101828083C701E55A
:1079400089EB938701E5D84318C188473E953105F7
:10795000828001458280938701E523A207000547C5
:107960002380E7008280938701E5A380A7008280BF
:10797000814629A8130777052380E50035A0938762
:107980007705A380F50089050505850663F6C6021F
:107990008347050013D74700BD8B2548E36CE8FCFF
:1079A000130707032380E5002547E36AF7FC938765
:1079B0000703A380F500C1BF8280011106CE230614
:1079C000A10093578500A306F100935705012307F3
:1079D000F1006181A307A10011466800EFF05FF993
:1079E000F2400561828081461DA813086004636926
:1079F000F804938797FC93F7F70F2A97034717002C
:107A0000130890036363E804130707FD1377F70F68
:107A100092073388D500D98F2300F800850663F4D8
:107A2000C60413971600B307E50083C707001308C1
:107A30009003E36CF8FA938707FD93F7F70F75BF90
:107A4000938797FA93F7F70F4DBF130860046367A6
:107A5000E800130797FC1377F70F5DBF130797FA3A
:107A60001377F70F75B78280011106CE22CC2E84D2
:107A700011466C00EFF03FF78347C1000347D10088
:107A80002207D98F0347E1004207D98F0347F1004E
:107A90006207D98F1CC0F240624405618280814830
:107AA0008147814639A03388D5002300E800850648
:107AB000850763F6C7023307F5000347070013087D
:107AC000D007630C0701E38008FE3388D500134715
:107AD00007022300E8008148D9BF8548D1BF368519
:107AE0008280411106C693874126238AA700EFD0E2
:107AF000EFB3B24041018280411106C68D45014578
:107B0000EFF03FD9B24041018280411106C6130611
:107B10000040B72500089385050693874126884BCA
:107B2000EF1030368D450945EFF0BFD6B240410128
:107B30008280411106C622C413844126AA863726B4
:107B4000000813068605930500400848EF10D02171
:107B50000848EF10302F8D45EFF0BFD3B2402244DC
:107B600041018280411106C622C41384412623109C
:107B70000400231104002312040023130400014510
:107B8000EFF03FF6A30A0400B24022444101828094
:107B9000011106CE93874126884734007000B7252F
:107BA0000008938545E87D05EF10F02222479307F2
:107BB000004063F3E7003EC4EFD09F94B2471D8DB1
:107BC000A24763EEA7022AC4938741269C4B130762
:107BD000C0062380E700EFD01F92938741269C4B7D
:107BE0002246B245AA9513851700EF1090298D45BE
:107BF00022450505EFF0FFC9F240056182809387B9
:107C000041269C4B1307D0062380E700E9B70111FA
:107C100006CE93874126884734007000B7250008B8
:107C2000938545E85D05EF10101B22479307004040
:107C300063F3E7003EC4EFF0DFACB2471D8DA2470F
:107C400063EEA7022AC4938741269C4B1307C00604
:107C50002380E700EFF05FAA938741269C4B2246E2
:107C6000B245AA9513851700EF10B0218D45224526
:107C70000505EFF01FC2F24005618280938741261F
:107C80009C4B1307D0062380E700E9B7397106DE65
:107C900022DC26DAB727000803A387EE938787EE56
:107CA00083A8470003A88700C8478C4BD04B944F4C
:107CB000D84F1AC646C842CA2ACC2ECE32D036D2A7
:107CC0003AD483C707022306F1029387412683D75C
:107CD000470013075014638CE7061307D014638E14
:107CE000E70A99CB93874126239207000D45F2506E
:107CF0006254D254216182801305F102EF1060209A
:107D000029CD938741269C4B1307F0042380E7007D
:107D10000144938741268C4B931714008507054631
:107D2000BE951305F102EFF0BFC405041305F1027F
:107D3000EF10201D79FD131514008D450505EFF09A
:107D40005FB593874126130750142392E700EFF0A5
:107D50003FB39387412688CB41C9138441265044C1
:107D60006916058250D0084493048402A68519053B
:107D7000EFF07FC75C503E94230404021546B725FC
:107D80000008938585ED2685EF10F00C0DE19387B3
:107D900041261307D0142392E700EFE01F90854798
:107DA00063E4A7000145A1B7EFF03FD625BF114618
:107DB000B7250008938505EE138541261305850236
:107DC000EF10700901E5EFF05FD429BF1306000240
:107DD000938741268C4B6800EFF09FB98D451305C2
:107DE0000004EFF01FABFDBD014511B7938741269D
:107DF00083D7270095EF411106C63D46B7250008F9
:107E0000938505E7938741268847EF10D00411ED4D
:107E1000EFF0BFCF0545EFF01FB5938741262391C3
:107E200007000D45B24041018280EFF0FFCCF5B76D
:107E300093874126239107000D4582809387412631
:107E400083D72700CDEF011106CE22CC93874126A0
:107E5000884703441500930770066302F4029307F2
:107E60007004630EF4009307D006630AF4009307CE
:107E7000D0046306F40093073006631FF406700015
:107E8000B72500089385C5E60905EF10C074EFF02B
:107E9000DFC70317C100930770066303F40293075B
:107EA0007004630CF4029307D006630DF402930789
:107EB000D004630EF402938741262392E74C29A055
:107EC00093874126239EE74A938741262391070003
:107ED0000D45F24062440561828093874126239FCD
:107EE000E74ADDB7938741262390E74CF1BF93879C
:107EF00041262391E74CC9BFEFF01FC0F1B793872C
:107F00004126239107000D4582809387412683D720
:107F1000270099C793874126239107000D4582804A
:107F2000411106C613060040B72500089385C5F029
:107F300093874126884BEF10C0748D450D45EFF0B7
:107F40005F9593874126239107000D45B24041017B
:107F500082809387412683D7270099CB1307B01AD5
:107F6000638EE70093874126239107000D458280A9
:107F7000938741261307B01A2391E700411106C6E3
:107F800022C41385412613050543EFE0EF9385478F
:107F900063F4A70401449307000263C18702938737
:107FA00041268C4B931634001307C4100A07BA9766
:107FB000B6958843EFF07FA00504F1BF8D4513050A
:107FC0008010EFF01F8D93874126239107000D4508
:107FD000B2402244410182800145DDBF411106C605
:107FE00022C49387412683D7270091CF1307501CC3
:107FF0006385E70493874126239107000D45B2402E
:1080000022444101828001449307000263C1870238
:108010009387412688471317340005079305C4103A
:108020008A05BE953A95EFF03FA40504F1BF93870A
:1080300041261307501C2391E700138541261305A1
:108040000543EFE04F92854763E4A700014545BF34
:10805000EFF0BFAB45B7411106C622C49387412656
:1080600083D7270091CF1307701D638BE702938797
:108070004126239107000D45B240224441018280F0
:108080001384412608441306844BB72500089385C2
:10809000C5E60505EF1020549307701D2311F40069
:1080A000138541268325854B1305454BEFE06F95DE
:1080B000854763E4A7000145C1B7938741268C4BF0
:1080C00003A5474BEFF07F8F8D452145EFF06FFC07
:1080D00079BF411106C622C49387412683D7270062
:1080E00091CF1307101F6386E704938741262391DE
:1080F00007000D45B240224441018280138441268D
:1081000008441306844BB72500089385C5E605058A
:10811000EF10604C08449305D0030505EF10E050C4
:108120009305444B0505EFF03F949307101F23116F
:10813000F4009387412683A5874B03A5474BEFE0C7
:108140000F9E854763E4A70001456DB7EFF0FF9BE5
:1081500069BF011106CE22CC26CA4AC84EC69387F3
:10816000412683D727008DC3130700216389E706C3
:1081700093874126239107000D45F2406244D24483
:108180004249B24905618280138441260444850432
:108190009305C0022685EF10404993091500130688
:1081A0000402372900089305C9E62685EF10A0428E
:1081B000130644029305C9E64E85EF10C04158509E
:1081C0009307004063F7E7009387412613070040B9
:1081D000D8D393874126130700212391E700138505
:1081E000412650510C5113058502EFE0CF9F854782
:1081F00063E4A700014551B71384412650500C4851
:1082000013058402EFF0CFF648508D450605EFF0D8
:108210004FE8B9BF411106C622C49387412683D7D0
:10822000270091CF1307C0226385E7069387412675
:10823000239107000D45B2402244410182801384FE
:10824000412608449306440213060402B725000899
:10825000938545E80505EF10003808449305A00311
:108260000505EF10803C050558509307004063F763
:10827000E7009387412613070040D8D31384412693
:10828000505093058402EFF00FF69307C02223119C
:10829000F4001385412650510C5113058502EFE07F
:1082A000CFA8854763E4A700014571B7EFF0FF85CC
:1082B000B5BF9387412683D7270099CB1307D024D6
:1082C000638EE70093874126239107000D45828046
:1082D000938741261307D0242391E700411106C656
:1082E000EFE06FDF854763E6A7000145B24041013B
:1082F00082800545EFF0EFFE93874126239107002A
:108300000D45EDB79387412683D7270099CB1307F7
:10831000C025638EE70093874126239107000D4512
:108320008280938741261307C0252391E7004111DE
:1083300006C6EFE02FE9854763E6A7000145B24096
:10834000410182800545EFF0CFF9938741262391C3
:1083500007000D45EDB7011106CE22CC93874126CB
:1083600083D7270091CF130740276384E7049387BF
:108370004126239107000D45F24062440561828049
:1083800013844126580034007000B72500089385F7
:10839000C5F40844EF102024B2472324F44CA2472C
:1083A0002326F44C92472328F44C930740272311AB
:1083B000F400938741269386474D03A6074D83A576
:1083C000C74C03A5874CEFE01F8F854763FDA700CF
:1083D0009387412603A5474D01E5EFF00FF341BF19
:1083E000EFF02FF569B7014541BF011106CE22CC50
:1083F0009387412683D7270091CF130700296384F1
:10840000E70493874126239107000D45F24062441B
:108410000561828013844126580034007000B7251E
:108420000008938505E80844EF10E01AB2472324BA
:10843000F44CA2472326F44C92472328F44C93078C
:1084400000292311F400938741269386474D03A604
:10845000074D83A5C74C03A5874CEFE08FE5854703
:1084600063FDA7009387412603A5474D01E5EFF083
:10847000CFE941BFEFF0EFEB69B7014541BF93870B
:10848000412683D7270099CB1307202A638EE70064
:1084900093874126239107000D45828093874126CB
:1084A0001307202A2391E700411106C6EFE02FB4FD
:1084B000854763FAA70093874126239107000D455E
:1084C000B240410182800145E5BF9387412683D7B1
:1084D000470099CB13074030638EE700938741260E
:1084E000239207000D458280938741261307403071
:1084F0002392E700411106C6EFF02F9A854763E605
:10850000A7000145B24041018280EFF00FE0938760
:108510004126239207000D45F5B7011106CE22CC66
:108520009387412683D76700130780346386E70467
:108530001307A0346384E70691CB938741262393E6
:1085400007000D45F2406244056182801305F10089
:10855000EF00301B65FD0545EFC09F890145EFF039
:108560004FD8138441268547A30AF400EFE05FCE7D
:10857000930780342313F400138541267105EFE03F
:108580005FCE854763F1A70A93874126DC4FB9E7A1
:10859000938741261307A0342393E700EFE02FA52C
:1085A000854763F4A7083725000813054502EF0047
:1085B000B012EFC00FEFEF0030123725000813059F
:1085C0004503EF007011EFF08F92EF00F0103725A8
:1085D000000813054504EF00301085B7094763868E
:1085E000E7020D47638AE70205476389E7003725FD
:1085F000000813054500EF00300E75B73725000859
:10860000130585F5EF00500D79BF372500081305D8
:1086100085F8EF00700C41BF37250008130505FDF4
:10862000EF00900B49B7014531BF014521BF411112
:1086300006C622C49387412683D727001307F00D6F
:10864000638AE70A1307500E6389E70691CB938785
:108650004126239107000D45B2402244410182800A
:108660009387412680472D46B72500089385C5E8A6
:108670002285EF00507E29C97D46B72500089385E5
:1086800085E92285EF00307D2DCD5D46B7250008B8
:10869000938585EB2285EF00107C3DC51946B725F3
:1086A0000008938505ED2285EF00F07A2DE1938790
:1086B00041261307500E2391E700EFF02FDD854789
:1086C000E3E7A7F8014549BFEFF0EFA9138441267E
:1086D00013060040B7250008938545060848EF00BB
:1086E000507A8D451305B004EFF0AF9A9307F00D63
:1086F0002311F400EFF07FE28547E3EAA7F4014598
:10870000A1BFEFF0EFC8A1B7EFF06FD089B7EFF0DE
:10871000AFBE35BF411106C69387412683D7670098
:108720001307B0366389E7021307C0366380E70496
:1087300089CB93874126239307000D45B240410121
:10874000828093874126DC4F9DE79387412613075C
:10875000B0362393E700EFE00F98854763FAA7024E
:10876000938741261307C0362393E700EFE09FB5B8
:10877000854763F1A702EFE0BFB80545EFF06FB69C
:1087800093874126A38A07000145EFC06FE655B7DE
:1087900001456DB701455DB7411106C69387412676
:1087A00083D7270089CF1307E0236382E7029387EB
:1087B0004126239107000D45B24041018280EFF030
:1087C000CFB4938741261307E0232391E700EFF00E
:1087D0007FF48547E3EDA7FC0145F9BF011106CE03
:1087E00022CC9387412683D747001307E02C63846C
:1087F000E7041307302D6388E70691CB9387412662
:10880000239207000D45F240624405618280138483
:108810004126084434007000B7250008938545E8D8
:108820003105EF00505BB2471CD0A2475CD09307E4
:10883000E02C2312F4009387412613868742CC5301
:108840008853EFE0DFAC854763F9A70293874126A1
:1088500003A5874205C1EFF0CFAD938741261307EB
:10886000302D2392E700EFF0FFEA8547E3E8A7F811
:10887000014551BFEFF06FA951B7014569B701112B
:1088800006CE22CC26CA9387412683D747001307FA
:10889000002F6382E7061307502F6388E70899CB00
:1088A00093874126239207000D45F2406244D2444B
:1088B000056182801384412608447000B7250008B2
:1088C0009385C5E63105EF001051B2471CD0044432
:1088D0009305A0031385C400EF00305505055044EF
:1088E000898C269693058402EFF06F9B48D09307FE
:1088F000002F2312F4009387412693868742138624
:108900008702CC538853EFE07FC3854763F9A70202
:108910009387412603A5874205C1EFF08FA1938776
:1089200041261307502F2392E700EFF0BFDE854763
:10893000E3E8A7F6014595BFEFF02F9D95B70145F8
:10894000ADB7011106CE22CC9387412683D74700CD
:1089500091CF13070032638BE7049387412623925C
:1089600007000D45F24062440561828093874126ED
:10897000DC4F85C301441305F100612311CD9387BA
:1089800041269C4BA2970347F1002380E700050492
:10899000DDB7EFF06F96D1B78D452285EFE07FEF21
:1089A00093874126130700322392E700EFF09FD60A
:1089B0008547E3E4A7FA014575B7411106C622C40D
:1089C0009387412683D727001307302B6388E70856
:1089D0006371F7021307502B6388E70A1307702BA4
:1089E0006393E702EFF0FFF5854763EEA7000145CB
:1089F00005A09DC31307102B6397E700EFF01FDE60
:108A0000854763FDA70A93874126239107000D45FB
:108A1000B2402244410182809387412680473146FB
:108A2000B7250008938505F12285EF00D04201E9C2
:108A3000938741261307102B2391E700C1B73146D6
:108A4000B7250008938505F22285EF00D04011ED8F
:108A5000938741261307302B2391E700EFF03FE285
:108A60008547E3E2A7FA014565B72946B72500081F
:108A7000938505F32285EF00103E11ED9387412683
:108A80001307502B2391E700EFF03FA48547E3EC59
:108A9000A7F60145B5BF3D46B72500089385C5F348
:108AA0002285EF00503B01E9938741261307702B85
:108AB0002391E70005BFEFF02F84B1B7014589BFCF
:108AC00083D741261307E00B636EF738011106CEFA
:108AD00022CC8A0737270008130707B7BA979C43A9
:108AE00082879387412683C75701639F070C13072B
:108AF00090092392E126EFE09FC59387412688C71E
:108B0000630C0534EFE07FD093874126C8C7130775
:108B1000C0092390E700EFE0BFD69387412688CBBA
:108B2000630E0532938741269C4783C70700A3073E
:108B3000F100130710076386E71A13071005638611
:108B4000E71C13078004638DE71C1307F00363849D
:108B5000E71E13077006638BE71E1307700463821A
:108B6000E7201307B0066389E72013073006638008
:108B7000E7221307D0066387E7221307D004638E2A
:108B8000E722130700076385E72413070005638CBA
:108B9000E724130730076383E7261307A007638AD8
:108BA000E7261307A0056381E7281307600763988A
:108BB000E7281307E00B2392E126EFF01FE085473B
:108BC00063EAA712014535AA9387412683C7470167
:108BD000E38F07F01305F1002D2639C9938741264D
:108BE0009C4B1307F0042380E70001449387412640
:108BF0008C4B9317140085070546BE951305F100AD
:108C0000EFE01FD705041305F100E52C65F11315FE
:108C100014008D450505EFE0DFC713071008239208
:108C2000E126EFE0FFC59387412688CB630005224C
:108C3000EFE0FFB19387412688C721CDEFE0FFBC6D
:108C400093874126C8C79C4703C707008D47631019
:108C5000F7048547631DF502130780082392E12678
:108C6000EFF0FF81854763F5A71E0145EFE07FE741
:108C700013060040B7250008938505059387412614
:108C8000884BEF0010208D450D45EFE09FC0EFE0D1
:108C90005FB89387412683C74701B9CF13071009EF
:108CA0002392E126138541266105EFD07FBC8547DD
:108CB00063F2A71A938741269C4F9DCF0145EFE0B1
:108CC0005FE213060040B7250008938545059387AA
:108CD0004126884BEF00F01A8D450D45EFE07FBB34
:108CE00021A81307000A2392E126EFF05F9485473D
:108CF00063F8A716EFE0FFB1130720072392E126E0
:108D00000545F2406244056182801307200A2392E0
:108D1000E126EFF0AF8D8547E3EEA7FC0145D5B71F
:108D20001307400A2392E126EFF04F918547E3E3D2
:108D3000A7FC0145F9B71307600A2392E126EFF07B
:108D4000CF9C8547E3E8A7FA014565BF1307800A72
:108D50002392E126EFF0EF9F8547E3EDA7F8014569
:108D60004DB71307A00A2392E126EFF02FA78547FE
:108D7000E3E2A7F8014571B71307C00A2392E12681
:108D8000EFF09FA18547E3E7A7F601459DBF1307D5
:108D9000E00A2392E126EFF0CFD18547E3ECA7F478
:108DA000014585B71307000B2392E126EFF06FBA58
:108DB0008547E3E1A7F40145A9B71307200B2392E8
:108DC000E126EFF02FC58547E3E6A7F2014515BF81
:108DD0001307400B2392E126EFF0EFA78547E3EB63
:108DE000A7F0014539BF1307600B2392E126EFF08E
:108DF0004FAE8547E3E0A7F0014521B71307800B8D
:108E00002392E126EFF00FD08547E3E5A7EE014579
:108E1000CDBD1307A00B2392E126EFF0CFD38547FA
:108E2000E3EAA7EC0145F1BD1307C00B2392E1264D
:108E3000EFF0AFDB8547E3EFA7EA0145D9B5EFE0F7
:108E4000BFCB4DBD239201260D4565BD014555BDE6
:108E5000014545BD014575B5014565B5014555B5AA
:108E6000014545B5239201260D458280411106C674
:108E7000EFB0DFE30D20EFB0DFC3EFE0BF8AEFE03C
:108E80007FCEEFB09FE83928EFB0BFC6EFB0BFD1BB
:108E9000EFF01FC3FDB79387C17323A0070023A280
:108EA000070082800D45828083A7C1731387170056
:108EB0009306F00F63D3E60001479386C173D44253
:108EC000638AE6009386C173B6972384A70098C28D
:108ED0000545828001458280411106C622C426C212
:108EE0002A8481440345040019C5EFF0FFFB01C546
:108EF00005048504C5BF2685B24022449244410141
:108F000082809387C173D8439C436306F70293879B
:108F1000C1733E97034787002300E500D843050748
:108F2000D8C39307F00F63DAE7009387C17323A2D6
:108F300007000545828001458280054582804111F8
:108F400006C622C42A844CC1EFB07FD308C0B24009
:108F5000224441018280411106C622C42A84EFB016
:108F60001FD21C401D8D05055C4033B5A700B240E3
:108F70002244410182800000000000000000000047
:108F80005D7106C012C216C41AC61EC82ACA2ECCEB
:108F900032CE36D03AD23ED442D646D872DA76DCD9
:108FA0007ADEFEC0F322103496C0F322003096C25F
:108FB000F322407C96C4732520348A85EF90AFBDA0
:108FC000864273901234964273900230A642739098
:108FD000427C82401242A2423243C2435245E245A1
:108FE000724682561257A2573258C258525EE25EFB
:108FF000725F864F61617300203000000000000046
:109000005D7106C012C216C41AC61EC82ACA2ECC6A
:1090100032CE36D03AD23ED442D646D872DA76DC58
:109020007ADEFEC073D0E87E7350F97E73D0B97ECD
:10903000F390D07E73700430B6427390427CA642A7
:109040007390123496427390223482401242A242AC
:109050003243C2435245E245724682561257A257E6
:109060003258C258525EE25E725F864F6161730091
:109070002030B687B2882A832E88639D061463F950
:10908000C50A4167636EE61AB70700016363F634E9
:1090900093568601E1471797FFFF1307A7013697FD
:1090A00003470700BA97130700021D8F19CB3398A7
:1090B000E500B357F500B318E60033E807013313B2
:1090C000E50013D608013355C80293960801C18202
:1090D000935703013377C802B385A602420733686A
:1090E000F700637AB80046989307F5FF63641801A8
:1090F0006367B8303E853308B8403357C80242032F
:10910000135303013378C802B386E602420833687A
:109110006800637BD80046989307F7FF63651801E2
:1091200079176363D8003E874205598D8145828057
:1091300001E60547B358C702416763EAE80EB7077F
:10914000000163ECF82893D68801E1471797FFFFE9
:10915000130747F6369783460700BE96930700022B
:10916000958FE5EB939E08013387154113DF0801C6
:1091700093DE0E018545935703013355E70333779B
:10918000E703B306D5034207D98F63FAD700C69722
:109190001307F5FF63E4170163E6D7263A85958F39
:1091A00033D7E703420313530301B3F7E703B30EC7
:1091B000D703C207B3E7670063FBD701C6979306DF
:1091C000F7FF63E51701791763E3D7013687420597
:1091D000598D828063E2D504C16763E2F604B70764
:1091E000000163E4F61E13D7860161489797FFFFDD
:1091F000938747ECBA9703C70700130E0002429704
:10920000330EEE40631A0E0C63EDB61C3335C50009
:109210001345150081458280814501458280930771
:10922000F00F63F3D71C13D786002148C1B713078B
:10923000F00FC686E37C17F193D68800A14739B7B3
:109240001307F00FB286E378C7E493568600A14770
:1092500099B5B398F80033D6D50013DF0801335E13
:10926000E6033397F500B356D500558F939E08015A
:1092700093DE0E013313F50093550701B376E60331
:10928000B387CE03C206CD8E63FBF600C6961306E7
:10929000FEFF63E4161763F2F616791EC6969D8EDE
:1092A00033D6E60393170701C183B3F6E60333858C
:1092B000CE02139706015D8F637BA7004697930745
:1092C000F6FF636817136376A7127916469793150E
:1092D0000E01098FD18D45B5B357E600B396C6018F
:1092E000DD8E33D3E50013DF0601B357E303939E0E
:1092F000060193DE0E013398C5013357E50033684C
:109300000701935808013316C6013373E303B3858D
:10931000FE024203B368130163FBB800B6981387DB
:10932000F7FF63EAD80C63F8B80CF917B698B3885E
:10933000B84033D7E803420813580801B3F8E803EC
:109340003383EE02C208B3E5080163FB6500B695FE
:109350001308F7FF63EDD50863FB65087917B69529
:10936000C207416FD98F1307FFFFB3F6E70093D809
:109370000701718F4182B38EE602B3856540B386E3
:10938000C60213D80E013387E802BA96C296338616
:10939000C80263F3E6007A9693D80601469663E224
:1093A000C5026385C5003E858145828041677D1782
:1093B000F98EC206B3FEEE003315C501F696E374CE
:1093C000D5FE1385F7FF8145828013D706014148FA
:1093D00031BD93560601C1477DB993D60801C147F7
:1093E000B5B38145054582803687014801B542877E
:1093F00085BF3E86E9BDBA871DBF328E4DB5791552
:109400004698D5B97915C69759BBB3C7A5008D8BBA
:109410003307C50081E78D4763EEC700AA876370F5
:10942000E50A83C6050085078505A38FD7FEE3EA15
:10943000E7FE828093763500AA8791CA83C605002D
:1094400085078505A38FD7FE93F63700FDB7937682
:10945000C7FF138606FE63F0C70683A3050083A239
:10946000450083AF850003AFC50083AE050103AEA1
:10947000450103A3850183A8C5019385450223A067
:10948000770003A8C5FF23A2570023A4F70123A652
:10949000E70123A8D70123AAC70123AC670023AEA5
:1094A00017019387470223AE07FF75B790419107D5
:1094B000910523AEC7FEE3EBD7FEE3E4E7F6828037
:1094C0003D432A876373C3029377F700BDEFADE591
:1094D000937606FF3D8ABA960CC34CC30CC74CC7A3
:1094E0004107E36BD7FE11E28280B306C3408A06D0
:1094F0009702000096966780A6002307B700A30690
:10950000B7002306B700A305B7002305B700A304DF
:10951000B7002304B700A303B7002303B700A302D7
:10952000B7002302B700A301B7002301B700A300CF
:10953000B7002300B700828093F5F50F939685005E
:10954000D58D93960501D58D61B793962700970227
:10955000000096968682E78086FA9680C1171D8F56
:109560003E96E374C3F8A5B735713ECBA6DA36C78D
:109570003AC942CD46CF9387418186DEA2DC84433F
:1095800063DB05009307B0089CC07D55F650665418
:10959000D6540D61828093078020231AF1002AC4DB
:1095A0002ACC814799C19387F5FF3EC83ECE74010E
:1095B000FD572E8426852C00231BF10036C2D92AA4
:1095C000FD576355F5009307B0089CC061D0A247D2
:1095D0002380070065BF71713ED39307402006C703
:1095E0002EC632CD36CF3AD142D546D72312F1021C
:1095F0002ACC2AD4812897070000938707033EDEF0
:10960000FD57B2452313F102938741812ACE2AD612
:10961000884334092E862C0882C682D036CAE129B6
:10962000BA404D6182800145828093F5F50F8347F2
:10963000050091C76393B70082800505CDBF91C136
:1096400001458280AA87850703C7F7FF6DFF338531
:10965000A7407D15828005C67D160147B307E5004A
:10966000B386E50083C7070083C606006396D7006C
:109670006304C7000507FDF33385D74082800145A9
:109680008280AA8709CA850503C7F5FF85077D166D
:10969000A38FE7FE65FB3E966393C7008280850734
:1096A000A38F07FED5BF01114AC803A9850022CCAC
:1096B00052C45AC006CE26CA4EC656C22E84328B1B
:1096C000368A63EE260983D7C50013F7074851C7CA
:1096D00004408C495848AA8AB389B4408D44B38465
:1096E000E4020947B3C4E402138716004E9763F3FC
:1096F000E400BA8493F70740D9C3A6855685EF10D6
:10970000003D2A890DE5B14723A0FA008357C40024
:109710007D5593E707042316F400F2406244D244D7
:109720004249B249224A924A024B056182800C4862
:109730004E86EFF09FCD8357C40093F7F7B793E7BA
:1097400007082316F4002328240144C84E99B38443
:1097500034412320240104C4528963732A015289AD
:1097600008404A86DA85EF1020271C440145B3875C
:1097700027411CC41C403E992320240179BF268622
:109780005685EF10A0422A895DFD0C485685EF10E2
:10979000402995BF83D7C500717126D34AD14ECFDA
:1097A00006D722D552CD56CB5AC95EC762C566C30D
:1097B00093F70708AA892E89B284B9C39C49A9E303
:1097C0009305000436C6EF1080302320A90023281B
:1097D000A900B24615E1B14723A0F9007D55BA5062
:1097E0002A549A540A59FA496A4ADA4A4A4BBA4BF5
:1097F0002A4C9A4C4D61828093070004232AF90079
:1098000093070002A30CF1029307000302DA230D71
:10981000F10236CE930B5002979AFFFF938A8A99F2
:10982000054C294B26848347040099C3639D77091F
:10983000B30C9440638E0C00E6862686CA854E855E
:10984000EFF07FE6FD576304F51AD256E69636DA56
:1098500083470400638D0718FD579304140002D05A
:1098600002D63ED202D4A301010682DC83C50400E5
:1098700015465685EF10A01413841400825731E565
:1098800013F7070109C713070002A301E10613F745
:10989000870009C71307B002A301E10683C60400CD
:1098A0001307A002638BE602B25726848146254641
:1098B0000347040093051400130707FD6374E606CD
:1098C0008DC63ED61DA00504B9BF330555413315DD
:1098D000AC00C98F3ED0A28451BF724793064700A7
:1098E000184336CE634907023AD60347040093076C
:1098F000E002631FF704034714009307A002631BF1
:10990000F702F2470904138747009C433ACE63C12C
:1099100007023ED235A83307E04093E727003AD646
:109920003ED0E1B7B387670385462E84BA9749B71F
:10993000FD57C5B7050402D2814681472546034736
:10994000040093051400130707FD6378E606F1F29F
:10995000834504000D461795FFFF13052586EF107C
:10996000000611CD9797FFFF938747851D8D9307BD
:109970000004B397A700025505045D8D2AD08345E6
:10998000040019461795FFFF1305858393041400FF
:10999000230CB102EF10A00225C59767FFF793874C
:1099A000676695E70257F2471377071009CF9107CB
:1099B0003ECED257D2973EDAB5B5B3876703854618
:1099C0002E84BA97ADBF9D07E19BA107D5B7780854
:1099D00097060000938666CD4A860C104E85970048
:1099E0000000E7000000FD572A8AE314F5FC8357C6
:1099F000C9007D5593F70704E39307DE5255C5B3BD
:109A0000780897060000938646CA4A860C104E8551
:109A10006D23D1BF411106C622C426C24AC0FD57DC
:109A2000639AF500FD54B2402244268502499244CF
:109A3000410182808357C60013F9F50F93F4F50FA7
:109A400093F7F7FD2316F6005C5A584285C71C5E53
:109A50003284635CF7001C401387F7FF18C0A38FA4
:109A600027FF5C4085075CC07DBFB285EF00306793
:109A70007DD14DBF144A1C4281CE63FBF60083C6E4
:109A8000F7FF63979600FD1705071CC258C261BF18
:109A90005CDE930746045CDA8D471CDE93076604A0
:109AA0001CC2854738C2230326055CC2ADBF4111E5
:109AB00022C42E84CC5906C69DC1930744046384F6
:109AC000F500EF0010763C40232A04025CC081CBF5
:109AD0005C5C01451CC0B2402244410182801C48AC
:109AE000232204007D551CC08357C40093E707025E
:109AF0002316F400CDB7130101D297070000938716
:109B0000A7F12326312D232CF1289309C1019707B2
:109B10000000938707FA232C812C232A912C2328D9
:109B2000212D2324412D2322512D2320612D232E4D
:109B3000712B232C812B232E112C232A912B2328AC
:109B4000A12B2326B12BAA842E84232401122326A1
:109B5000011223283113232EF12836CC130A500288
:109B6000130BA002A54B2949978AFFFF938A0A6528
:109B7000176CFFF7130C0C498347060032C6638548
:109B80000732EF00B05E3246834D0600930C16009C
:109B90006E9583471500A18BB1C35C406359F002F9
:109BA000EF00D05C1C4003C707003A95034715003F
:109BB000218B19E36686C9B70327C11285071CC02C
:109BC00005072326E11258407D1758C0F9B78327AF
:109BD000C129A2852685829761D5E9BF639A4D1771
:109BE00023220112232E0110834716006397670179
:109BF000C147232EF110930C260083C50C00668DFF
:109C0000850C938705FD63F0FB060D465685EF0036
:109C1000105B01CD330555418547B397A700032558
:109C2000C111668D5D8D232EA11083470D00130792
:109C30007006930C1D006366F7081307500663F067
:109C4000E71C13077004636AF7021307500463F8F4
:109C5000E71A638B0712638D470F8D47232AF11292
:109C60002320211361A083274112B307F9029387B0
:109C700007FDAE972322F11249B71307B00563839E
:109C8000E7126365F70213078005E398E7FC0327F3
:109C9000C11113670720232EE11041472320E11251
:109CA0001307E006B337F7008D073DA8130730060A
:109CB0006387E71013074006E391E7FA2320211397
:109CC000C5B7130700076383E70C6365F70613073F
:109CD000E006638FE70E6362F70C13079006E39EBE
:109CE000E7F6232001128D47232AF1125C40635AC4
:109CF000F0108327C11193F7070481EFEF0010479D
:109D00001C4003C707003A9503471500218B6312D7
:109D100007108327411309476342F712340822864C
:109D20006C0A2685352B85476300F5188947E313B0
:109D3000F5E881A813075007E382E7F813078007C7
:109D4000E387E7F413073007E399E7F0894769BF32
:109D50005C406352F0021C4003C707006316B7154E
:109D6000850758401CC08327C1127D1758C085073E
:109D70002326F11281B58327C129A28526858297E2
:109D800079D90325811279ED7D55D5A00327C1111D
:109D900013670702232EE110DDBDA1472320F11236
:109DA000914799B7E6854E85EF0030008327C111B2
:109DB000AA8C93E70704232EF110854735B7832734
:109DC000C111232A011293E70704232EF11039BF92
:109DD0008327C11113F70701E31E07DC624793F5E0
:109DE00017008326C1121306470091C532CC1C43CD
:109DF0002390D700C1B332CC1C4394C365BB9547B5
:109E0000E5B58327C129A28526858297E30305EE60
:109E10008DBF0327C11205072326E11258407D1785
:109E200058C06355E00085071CC0C9BD8327C12900
:109E3000A28526858297E30305ECA1B71147634805
:109E4000F700340822866C0A26850123E9BDE30366
:109E50000CD6340822866C0A268597000000E7009D
:109E60000000D1B58357C40093F7070491FF832006
:109E7000C12D0324812D8324412D0329012D832904
:109E8000C12C032A812C832A412C032B012C832BE8
:109E9000C12B032C812B832C412B032D012B832DD4
:109EA000C12A1301012E828003258112C9B779715D
:109EB00056CA9C49BA8A984522D426D24ECE52CC54
:109EC00006D64AD05AC85EC6AA892E84B284368A7B
:109ED00063D3E700BA879CC00347340419C38507DE
:109EE0009CC01C4093F7070281C79C4089079CC017
:109EF0000329040013796900631A0900130B940104
:109F0000FD5B5C449840998F634CF9041C40834688
:109F1000340493F70702B336D000A5EB13063404DC
:109F2000D2854E85829AFD576303F5041C40114685
:109F30009840998B544481446397C700B384E640AA
:109F400063D3040081441C4418486354F700998F7C
:109F5000BE94014969047D5B63982405014509A805
:109F600085465A86D2854E85829A631E75017D5537
:109F7000B250225492540259F249624AD24A424B98
:109F8000B24B456182800509ADBF3307D40013068B
:109F90000003A301C7040347540493871600A29744
:109FA0008906A381E7049DBF85462286D2854E851A
:109FB000829AE30E65FB050945B7797122D426D252
:109FC0004AD04ECE06D652CC56CA5AC8B68983C697
:109FD00085019307E0063289AA842E84138635040E
:109FE0006381F61E63E2D706930730066382F60AA2
:109FF00063EDD700638B061E930780056387F61613
:10A00000930A24042301D40469A8930740066386B5
:10A01000F60093079006E395F6FE1C40084393F67E
:10A02000070893054500C1C21C410CC363D8070053
:10A030001307D002B307F040A301E4049786FFFFA3
:10A0400093868618294765A0930730076383F61A1D
:10A0500063EFD7009307F006638FF60493070007BA
:10A06000E390F6FA9C4193E707029CC109A8930785
:10A0700050076382F60493078007E393F6F893078B
:10A080008007A302F4049786FFFF93862615E5A0B8
:10A090001C43938A2504938647009C4314C3238161
:10A0A000F5048547BDA293F607041C410CC3BDDE31
:10A0B000C207C187A5BF0C401C4313F805081385D0
:10A0C00047006305080008C39C4339A093F50504C5
:10A0D00008C3FDD983D707001307F006638BE60C8E
:10A0E0009786FFFF9386460E2947A30104044C4040
:10A0F0000CC463C5050008406D9908C099E3B28A95
:10A1000091CDB28AB3F5E702FD1AB69583C5050075
:10A110002380BA00B3D5E70263F3E70AA147631EC1
:10A12000F7001C40858B91CB58401C4863C7E70063
:10A1300093070003A38FFAFEFD1A3306564110C899
:10A140004E87CA867000A2852685EFF05FD67D5ABD
:10A150006315450D7D55B250225492540259F2496F
:10A16000624AD24A424B45618280A382D5049786D7
:10A17000FFFF938666050C40084313F805081C4151
:10A1800011056300080208C313F7150001C793E522
:10A1900005020CC04147B1FB0C4093F5F5FD0CC026
:10A1A000A9B713F8050408C3E30008FEC207C1837A
:10A1B000E1BF9786FFFF9386260121473DB7AE8713
:10A1C00091B794411C43CC4913F806081385470006
:10A1D0006306080008C39C438CC301A808C393F618
:10A1E00006049C43F5DA2390B70023280400B28AC2
:10A1F00081BF1C43D04181459386470014C383AA85
:10A2000007005685EF00A07B01C53305554148C0C6
:10A210005C401CC8A301040425B714485686CA85AF
:10A2200026858299E30845F31C40898B8DE7B24768
:10A230004844E352F5F23E8539BF85465686CA85C5
:10A2400026858299E30865F1050A5C443247998FB7
:10A25000E345FAFEE9BF014A930A94017D5BF5B735
:10A260009C45011122CC26CA52C406CE4AC84EC60D
:10A2700056C25AC02A8A2E84B28491E7984D8547E7
:10A2800011C3FD571CC41C40C18B99E79C42138726
:10A29000470098C283A907000149854A094B084C29
:10A2A0001DC5631255099C4003C707005C48BA9757
:10A2B00083C7070089EF63180904F2406244D2445F
:10A2C0004249B249224A924A024B056182801C40AF
:10A2D0000509C18B99E79C40850983C70700A38FB7
:10A2E000F9FE9840DC40050798C01844FD17DCC013
:10A2F0007D1718C409CBE344F0FA83270418A68518
:10A300005285829749DD1C40C18B81EB5C448507F7
:10A310005CC41C4C99C3238009001C4801453E992C
:10A320002328240159BF631B650189259C4083C7ED
:10A3300007003E9583471500A18BD1DBE31509FC8F
:10A34000084C8547E311F5FC8DBF5D719787FFFFD2
:10A35000938747EBCAC03EC236899787FFFF938732
:10A36000A7EA944D3EC49787FFFF938727EAA2C4CC
:10A370004EDE5AD86ECE3EC686C6A6C252DC56DA2D
:10A380005ED662D466D26AD08D47AA892E84B28DF9
:10A39000170B0000130B8B536396F600170B00008E
:10A3A000130BEB3D1C449306C015014A1386F7FFBF
:10A3B00063F7C600138A37EA9307D0151CC41C4004
:10A3C0008566938606D09304C401D58F1CC0130CF8
:10A3D0004100A68A814B930C002083A70D00032522
:10A3E0000C00094683C50700D92B25C1854763901A
:10A3F000FB0E5C4099E71C40214758C093E70720BB
:10A400001CC01C4093F7F7AF1CC01C441386F7FF19
:10A4100010C485CF03A60D00138D1A0093071600F4
:10A4200023A0FD00034606002380CA0003A64D00BA
:10A43000EA8A7D1623A2CD006349C00003260418D2
:10A44000EE854E850296631A0510850B8D47110C1B
:10A45000E395FBF85C4099E3A9475CC05C40484841
:10A460009785FFFF9385C5D99D8DFD7B056C568D26
:10A470002D2A814A930C0003938BFB6F130C0C80E5
:10A4800014441040C9C203A50D004C480348050000
:10A49000C29583C50500A5C963189805B3758601E3
:10A4A000A1C5850A63050A0085067D1A14C483A622
:10A4B0004D00FD1623A2DD006351D00483A60D00DC
:10A4C000850623A0DD001444FD1614C455BF89473A
:10A4D000E39DFBF21C4013F60760E31896F7414733
:10A4E00058C093E707100DB73376760110C0834646
:10A4F0000500050DA30FDDFE5DBF83260418EE8564
:10A500004E85829669D1144093F6061085C263FC8D
:10A51000A4018345FDFF8326C417130AFDFF6E8641
:10A520004E858296528D0545630F9D041840418BE0
:10A5300021E723000D0054400146A6854E85029B6D
:10A5400014400327090013F6060211CA93064700B8
:10A550002320D900184308C329A8814A6DB793F571
:10A560001600130647009DCD2320C9001843231071
:10A57000A7005844050758C41C48B3049D40D6940E
:10A58000BE9404C80145B640264496440649F25993
:10A59000625AD25A425BB25B225C925C025DF24D1F
:10A5A000616182802320C90075B783C70500130746
:10A5B000E0056388E704138715008146014693058B
:10A5C00000103308C5002300D8000506E31BB6FEC3
:10A5D0001306F7FF8DC793C616009308D002130821
:10A5E000D0053306F5002300D60083450700130687
:10A5F0001700638415036384050191E93A86328567
:10A6000082801387250083C71500854645BFAE8726
:10A610003287C1BF9307D002E5BF83451700E38BA4
:10A6200005FFE3C9F5FE090785073306F50023009A
:10A63000D600E3CBB7FE55BF79714AD04ECE06D6D1
:10A6400022D426D2AA892E899304190003C4F4FFC8
:10A650003A8536C632C42EC23AC031262295834787
:10A66000150002479245A18B2246B246C9E79307DF
:10A67000D0026314F40883C704000543930429003F
:10A68000FDC641476392E60213070003639EE7009D
:10A6900083C704001307800593F7F70D6394E70C55
:10A6A00083C71400C1468904B708008063140300FF
:10A6B00093C8F8FF33FFD80201480145A54FE54E86
:10A6C000FD5233DED802138707FD63E4EF04BA8737
:10A6D00063DFD704630D58007D58636AAE006314CE
:10A6E000AE006346FF0005483385A6023E9585040B
:10A6F00083C7F4FFC9BF268981BF9307B0026305F2
:10A70000F400A2870143ADBF83C70400930429006E
:10A71000D5BF1387F7FB63E5EE00938797FC4DBF2A
:10A720001387F7F963E5EE00938797FA55B7FD575E
:10A73000631FF8009307200223A0F900468519EE55
:10A74000B250225492540259F24945618280630406
:10A7500003003305A0406DD6630408009385F4FF21
:10A760000CC2F9BF93070003A1F2A14635BF13073E
:10A770000003E38FE7F0A94605BF938741819C431F
:10A78000985309E71767FF17130787D76FF0DFEABA
:10A7900079714AD04ECE06D622D426D2AA892E89E5
:10A7A0009304190003C4F4FF3A8536C632C42EC29E
:10A7B0003AC0552A22958347150002479245A18B3E
:10A7C0002246B246BDEF9307D002631EF40683C74C
:10A7D0000400054393042900F5C241476392E60251
:10A7E00013070003639EE70083C704001307800577
:10A7F00093F7F70D639FE70A83C71400C1468904E6
:10A800007D57335ED70201480145254FE54EB378A9
:10A81000D702138707FD6364EF04BA8763D1D706B5
:10A82000634D08047D58636AAE006314AE0063C6CE
:10A83000F80005483385A6023E95850483C7F4FFDA
:10A84000C9BF2689B1BF9307B0026305F400A28790
:10A85000014359B783C7040093042900D5BF138768
:10A86000F7FB63E5EE00938797FC4DBF1387F7F97D
:10A8700063E7EE00938797FA55B77D587DBF635F16
:10A8800008009307200223A0F9007D5519EEB2506D
:10A89000225492540259F2494561828063040300B4
:10A8A0003305A0406DD6630408009385F4FF0CC205
:10A8B000F9BF93070003A9F6A14699B71307000350
:10A8C000E384E7F2A9462DBF938741819C439853C7
:10A8D00009E71767FF171307A7C26FF07FEB011196
:10A8E00022CC2E84CC5906CE26CA4AC84EC652C4A3
:10A8F000930744046394F50493050040C92A11E9C1
:10A900007D55F2406244D2444249B249224A05612F
:10A910008280930700401CDC8347640448D81305F9
:10A92000D53F2301F50083475404A300F500834776
:10A9300044042300F50008C00145E1B7032984035E
:10A94000931919004E869D24AA845DD9330A2501E6
:10A95000AA854A865285EFE05FAB2320440144D8A4
:10A96000232C3403D1BF0325C50E828093874181F8
:10A970009C439C5389E79767FF17938767B803A5A4
:10A98000C70E828085E141116C00014511CA7955DD
:10A9900081CA834706009CC1034506003335A000E9
:10A9A00041018280014519CA795589CA8347060049
:10A9B0009CC1034506003335A0008280828093F558
:10A9C000F50F2A966314C500014582808347050070
:10A9D000E38DB7FE0505FDB763F3A504B386C50097
:10A9E000637FD5029345F6FF8147FD176393F5001A
:10A9F00082803387F600034807003387C7002A9711
:10AA000023000701DDB73387F500834607003307CE
:10AA1000F50085072300D700E317F6FE8280814703
:10AA2000E5BFCDC583A7C5FF411122C406C626C216
:10AA30001384C5FF63D307003E94AA84292C97672B
:10AA4000FF179387E7C59C4389EF2322040097678C
:10AA5000FF1723A787C42244B240268592444101B0
:10AA6000E5AA637EF40014403307D4006396E70040
:10AA70009843DC43369718C05CC0D1BFBA87D8432F
:10AA800019C3E37DE4FE94433386D700631F860039
:10AA90001040B29694C33386D700E31EC7FA104322
:10AAA0005843B29694C3D8C37DB76375C400B14709
:10AAB0009CC055B71040B306C4006316D7001443BA
:10AAC0005843B29614C058C0C0C371B782800111F8
:10AAD00026CA93843500F19806CE22CC4AC84EC6C9
:10AAE000A104B14763F7F404B14463E6B4042A89CE
:10AAF0009D229767FF179387A7BA98433A8431E45A
:10AB00009767FF17938707BA9C4381EB81454A8576
:10AB1000D5289767FF1723A7A7B8A6854A85DD2004
:10AB2000FD5963193507B1472320F9004A852D22C5
:10AB300029A0E3DC04FAB1471CC10145F24062449C
:10AB4000D2444249B249056182801C40858F63C06E
:10AB50000704AD4663F6F6001CC03E9404C001A88D
:10AB60005C40631487021767FF17232BF7B24A85EF
:10AB7000E5201305B4009307440061993307F540BD
:10AB800055DF3A94898F1CC055BF5CC3CDB722876F
:10AB90004040B5B7130435007198E30185FCB30557
:10ABA000A4404A858520E31B35FBB5BF81E5B2850E
:10ABB0006FF0FFF1011122CC06CE26CA4AC84EC65C
:10ABC000328401EEEFF0FFE50149F24062444A852C
:10ABD000D2444249B24905618280AE84AA89B5282F
:10ABE0002689E37485FEA2854E85EFF05FEE2A8903
:10ABF00069DDA6852286EFE05F81A6854E85EFF0B0
:10AC00005FE2E1B7411122C42A842E859777FF17AE
:10AC100023A607AE06C6EF702FF9FD576319F5009E
:10AC20009777FF17938787AD9C4391C31CC0B240B1
:10AC300022444101828091CD9307F00F63F7C70052
:10AC40009307A0081CC17D5582802380C50005455F
:10AC50008280014582808280828083A7C5FF138520
:0EAC6000C7FF63D50700AA959C413E958280F0
:04AC700000000300DD
:08AC7400400080000000000018
:04AC7C0003020102CC
:04AC800004030904BC
:10AC840009024300020100803209040000010202AB
:10AC9400010005240010010524010001042402021E
:10ACA40005240600010705820308000A09040100BF
:10ACB400020A0000000705030240000007058102A4
:10ACC40040000000FF000000DE48000818490008AA
:10ACD400C8490008764900084449000800000000FB
:10ACE4000000000000000000000000000000000060
:10ACF4000000000000000000000000000000000050
:10AD0400000000000000000000000000000000003F
:10AD1400000000000000000000000000000000002F
:10B0F4000000000000000000000000000803000839
:10B1040000000020000000001C03000800000000F4
:10B11400000000000000000000000000000000002B
:10B124002C2200084C2200080C2200080000000019
:10B13400000000000000000000000000000000000B
:10B1440000000000000000000000000000000000FB
:10B1540000000000000000000000000000000000EB
:10B1640000000000000000000000000000000000DB
:10B174000000000000000000000000004300000088
:10B1840000000000000000000000000000000000BB
:10B194000000000000000000000000004300000068
:10B1A400000000000000000000000000000000009B
:10B1B4000000000000000000000000004300000048
:10B1C400000000000000000000000000000000007B
:10B1D4000000000000000000000000004300000028
:10B1E400000000000000000000000000000000005B
:10B1F4000000000000000000000000004300000008
:10B20400000000000000000000000000000000003A
:10B2140000000000000000000000000043000000E7
:10B22400000000000000000000000000000000001A
:10B2340000000000000000000000000043000000C7
:10B2440000000000000000000000000000000000FA
:10B2540000000000000000000000000036AC000800
:10B2640084A90008000000007C220008782200085D
:10B27400081F0008081F0008081F0008081F00080E
:10B28400081F0008081F0008081F0008081F0008FE
:10B29400081F0008FFFFFFFFFFFFFFFFFFFFFFFF87
:10B2A400FFFF000001004153434949000000000032
:10B2B400000000000000000000000000000000008A
:10B2C4000000000000004153434949000000000011
:10B2D400000000000000000000000000000000006A
:10B2E400000000000000000000170020FF00000024
:10B2F40000C2010000000800010100009C040020BD
:08B30400000000000102030437
:040000050800015C92
:00000001FF
